:020000041100E9
:10300000002373B52B4D2C4C28006361022601F080
:1030100065FA4021FE2221742800284B009601F019
:10302000AFFA002836D1217CFF222800244B0096DD
:1030300001F0A6FA00282DD1224BA2899A4226D16E
:10304000E389214A93420DD1204B6361204B2268D2
:10305000002A03D1002B01D043CB43C4280001F048
:103060007BFA73BD1B4A934201D00023EFE71A4B52
:103070001A4A1B68934206D9C02304222800217CE7
:103080009B0001F0F3FA114B6361154BDFE700235E
:103090002374EAE7CC233821AC2228009B01217459
:1030A00001F0E4FA0028F2D10E4B63610E4BE3818C
:1030B0000E4BCCE7BC44FF1F6C64FF1F7864FF1FFE
:1030C0007A64FF1F5959000083050000094300116D
:1030D00024BF0011821500009064FF1F87130000B9
:1030E00030BF0011C1430011AAAAFFFF18BF001191
:1030F000F7B5164B0192C318021D002000938823D8
:103100005B05D3181B685C1C1AD09CB2402C18D8E5
:103110008D781E0CAC466746CD782D023D43AE42FD
:1031200006D1019800280ED110000C70240A4C70B2
:1031300003249BB20733A343D218009B9A42DED3E9
:10314000FEBD4432F9E71000FAE7C046FC0F00006C
:10315000802213B503000324019189B25201073183
:103160009B18A14304305A1A88235B05C3181B68B7
:10317000591C03D190429241104016BD99B240298A
:1031800007D80B000733A343C0189042ECD30020AC
:10319000F3E74430F9E7134B134A1B68126810B584
:1031A000FA24934201D81A00F824104BE4021B6859
:1031B0009A4210D813000E4A12689A420ED3013375
:1031C00007D1F823DB029C4203D10A49054808F0E5
:1031D00027FE200010BDFC24E402ECE7FE24E402FC
:1031E000F7E7C04600C0071100D0071100E0071143
:1031F00000F00711FFFFFF7FF0B59BB015000490B2
:103200000391402A00D9A0E006AB59801A80FFF74D
:10321000C2FF0400042816D9002206A9FFF768FFA0
:10322000052810D906AB1B88AB420CD1002D07D066
:10323000514B2A000499C01808F05AFD002802D109
:1032400001201BB0F0BD06AB1D8020000699FFF7E2
:103250007FFF041E7BD1069B0793FFF79CFF802313
:103260005B01C618802307001B039E4201D3F8268A
:10327000F60288235B05F31801931B68013302D023
:10328000019808F0CDFA3D49019808F0C9FD3B1DB1
:103290000293331D05938822029B52059B181B68DD
:1032A00008935A1C3CD044219AB20091402A04D879
:1032B0000320D11D814389B2009103991B0C8B42DD
:1032C00024D0402A22D80122300008A9FFF710FF9D
:1032D000021E1BD1380008A9FFF70AFF04000428CA
:1032E00031D9009A059B9B1880225201B218934253
:1032F00040D288235B05C118009A09A808F040FC59
:103300001D4B009A09A9F01808F0F2FB009A029BE5
:103310009446634402931A4B029AFB189A42BAD31A
:1033200088235B05FC1821680198013908F078FDB5
:10333000200008F075FA039A07AB5A80300007990D
:10334000FFF706FF0400002C03D1002079E70428D2
:10335000FBD988235B05E018069908F061FD03237B
:10336000EA1C9A4300D16BE7034B0499E01808F07C
:10337000BFFB65E70424ECE704000011FFFFFF7FBB
:10338000F80F0000F7B505001400402A21D80027E7
:1033900001AE71803780FFF7FEFE042816D93A008F
:1033A0003100FFF7A5FE042810D93688BC420BD0A7
:1033B000BD4209D0221CB44200D9321C064B92B245
:1033C000C118280008F0DCFB30B2FEBDC04300B2DB
:1033D000FBE703204042F8E70400001137B5042260
:1033E00004000D0001A81649FFF7CCFF02000428D5
:1033F0000BD1019BA34208D3AB4204D0104901A8D2
:103400000195FFF7F9FE01203EBD0E4C2368200018
:10341000019308F005FA019920000139019108F0A3
:10342000FFFC80235B01E418074B9C42EED1042291
:10343000034901A80195FFF7DFFE0020E4E7C0463D
:103440005555000000C007110000081130B589B0C3
:1034500008F06EFC10226946254808F0A1FB254BB8
:10346000009A9A420ED1019B029A0F2B33D8002169
:1034700001240698013B08D2002900D00292029B49
:10348000013331D10023029325E0551CF2D1020013
:103490002100EFE710341022200004A908F080FB7F
:1034A000029B013301D1069B0293882304995B059B
:1034B000C918059B06981A03120B049105928142C4
:1034C00003D02B4201D108F05BFB019B013B019330
:1034D000019B002BDED1029B002B03D004930498A8
:1034E0004168084709B030BDE025014C2D03EFE7E6
:1034F0000000011150485936F7B50F4F0F4BFA6DC8
:1035000004001A4084235B001343FB65030010335F
:10351000019300252E00112008F04AFA0322BB6E09
:103520001340AB4002351E43202DF4D1019B40C413
:10353000A342EED1F7BDC04600F0004000FEFEFF02
:10354000802270B5AD4CAE4BD200002120001C6033
:1035500008F086FA2300AB4A88331A60AA4B1A781F
:103560006E23002A00D01133E3620A232365A74BA0
:103570001878A74BA0630138E361C3B2032B01D8CD
:1035800010232362A34B37226361C823DB00A361AE
:1035900023008C331A60082336210F3AE518E163C3
:1035A00023646264E9670439251DE96725003B2629
:1035B000BC352E602500C0352B602500C4352A603F
:1035C00025000636CC352E602500083EC8352E6015
:1035D0002500D03529602100D4310B602100D8317D
:1035E0000A6021000225E0310D6025004221DC3512
:1035F000296025001B3EE4352E602500E8352B6050
:103600002500EC352A6022000525F43215602200E1
:10361000F032116022001831903211602200943291
:10362000136023003C2298331A60AF23DB00236031
:10363000794B2363032805D808F0FAF833023537AD
:103640001523636096232100FA225B00A360E360E8
:10365000C8332361714BFC319200A3640A6062623B
:103660006F4A704DA2627322E2656D3A6265A2658F
:103670000232E5644A600221616696218900A166F2
:10368000626709210022E166A2676749674A684EBE
:103690002167E2673560032811D808F0C9F8960859
:1036A0009EA61023CDE70E23CBE70C23C9E720000D
:1036B0001A259C30056020000735A03005602000E9
:1036C000A83003602300FA20F8338000186023003C
:1036D0006420A433186023005F38AC3318602300E3
:1036E0000338B03318602300C630B43318602300A9
:1036F0000020B833186023003825FC339D604D4D01
:103700005A665D644C4D9A64DD619625AD001D627C
:103710004A4D9A675D62F53DFF3D9D621E25484A10
:10372000DD6618675867D9651966DA67BE23C02158
:10373000444A5B00E250444B4900635004316250FC
:10374000C4225200A350FA23E4205B000432A350A9
:103750000432A3503D493E4A3E4BD1603E49800071
:1037600019503E49E938FF3819503D490430195085
:103770003C491038D1613C4911633C4951633C4993
:1037800011603C49195019003B48F83108603B4929
:10379000D16582213A4A89005A501A0039490832C3
:1037A000D1671A003849B43211608821374A89003C
:1037B0005A501A00364988321160364ADA6408F0E5
:1037C0005FFA012008F0FCF970BD200014259C3040
:1037D000056020000435A03070E7200010259C30E3
:1037E000056020000335A03068E720000E259C30DE
:1037F000056020000235A03060E7C0460004FF1FCE
:103800004467FF1F3072FF1F0047FF1F4A0AFF1F58
:103810003A07000080C3C9019A02000050C30000AB
:103820006A180000280A0000204E000088130000DB
:10383000F009FF1F001F001168100000C4090000FC
:10384000DC05000040420F0010270000FD1BFF1F99
:10385000FC00FF1F0000FF1F012FFF1F2932FF1F69
:10386000C130FF1FD51FFF1FF11FFF1F9D21FF1F2D
:10387000491FFF1FC128FF1F692CFF1FD918FF1FF9
:10388000CD27FF1F3525FF1F4125FF1F491EFF1FA5
:10389000011FFF1FC11DFF1FF7B50B0CFF270122E2
:1038A000009300233C001E001D009446019089B245
:1038B00062469A401000084018413618B6B2FF2FF1
:1038C00002D1012E00D19FB2009802401A41AD18DA
:1038D000ADB2FF2C02D1012D00D19CB20133102BCF
:1038E000E6D10320012E07D1012D04D1019B240133
:1038F000E4191C700138FEBD102EFCD10238102DC9
:10390000F9D00230F7E710B5064C2378002B07D129
:103910000548FFF7F1FD0548FFF7EEFD0123237091
:1039200010BDC0460567FF1F1867FF1F0867FF1F10
:10393000F0B58BB00D0001230190102936D8FFF7A8
:10394000E2FF00231A001B48C15C01335218102B00
:10395000FAD1023B002A29D0174B184C1F680023CC
:1039600006A9E25C1600FA5C56405E540133102B47
:10397000F7D102AA07F024FF2A0002A9019808F053
:10398000CFF908F0EDF823681B18236008F0E8F879
:1039900063681B18636008F0E3F8A3681B18A36052
:1039A00008F0DEF8E3681B18E360002318000BB092
:1039B000F0BDC0461867FF1FA045FF1F0867FF1F27
:1039C0000223F0B50124604D604E2B70604B91B026
:1039D0001C70604F0393336800212000BB7006F019
:1039E000D3FD200006F0CAFC0023984205D0BA7827
:1039F000552A02D0332A00D099E03360002006F027
:103A00002BFF08F0D5F9FFF79BFD07F0C9FE1F2239
:103A100001240021504B36261A70504B1C70504B1D
:103A20001970504B19689143163A0A431A60602284
:103A300019689143403A0A431A6007F051FF07F0B2
:103A40009FFFC120FF21484B80001A588A431A501B
:103A5000C522920098588843BF390143995098581D
:103A6000424908408021C90101438020995099585A
:103A7000C0050902090A0143995080213C484901C7
:103A800007F096FE0323220000933A4901943A4836
:103A900008F07EF82E22394904A808F071F802AB2C
:103AA00004ACF61861782078023406F087FCA64250
:103AB000F8D1334C334B226803201A40A023DB0299
:103AC00013432360802322689B04134323602268EE
:103AD0002D4B1A4080239B03134323602B4A2C4B0E
:103AE000934200D8012008F013F907F089FE8023E3
:103AF0002268DB0413432360287807F001FF039B4F
:103B00001878C0B208F03CF907F0CAFF2149042038
:103B100008F02EF806F06CFE00F0B6F800F0FCFDA0
:103B200000F08EFE00F01CFA002011B0F0BD0093F2
:103B30002100184A042008F043F98023DB059C6229
:103B4000FFF784FC5AE7C0464A0AFF1F34F00040E2
:103B50000047FF1F9C64FF1F480AFF1F490AFF1F01
:103B6000680AFF1FBCF0004000E100E0FF00FFFF1B
:103B70000447FF1F8859FF1F0457FF1F40BE001155
:103B800014F00040FF7FF8FFFFFF9FFF0080FF1F42
:103B90003072FF1F3B00010870B500252A492B4AEF
:103BA0002B484D6308CA1B051B0DED188242F9D145
:103BB0000022284B8B63284B08211A628022274B56
:103BC0009205DA67264BDA688A43DA60254A12786A
:103BD000012A03D09A6824490A409A6000260121EC
:103BE000224C11202660DA688A43DA6007F010FF61
:103BF000112007F025FE636C1D4A13406364EE2418
:103C0000E4006C431B4A200C0400642390420AD851
:103C1000FA223300D200904205D9174B0A21C0186E
:103C200007F02EFEC3B2154A11201372D48008F09B
:103C300047F8134B1B78002B04D1124B1021187836
:103C400007F036FF70BDC04600000540080605407D
:103C500080060540FF01000000F0004004E100E0A4
:103C60003CF000404A0AFF1FFFDFFFFF0038004022
:103C7000FFFEFFFFB70B000030F8FFFF8464FF1F5B
:103C8000BE66FF1FBC64FF1F002210B5110011208B
:103C900007F006FE10BD0000F8B500230125082638
:103CA000394F3A4C3B62E3681120AB43E360E36871
:103CB000B343E36007F0C4FD112007F0A9FE112013
:103CC00007F08EFF402322683000134323608023D7
:103CD0006268DB02134363608023A26802211343FE
:103CE000A360A3682A4A1340A3608023A2689B01B3
:103CF00013431022A360236C93432364236C2B4350
:103D0000236480231B013B62226B224B10271A4045
:103D10002263626B1A406263A26B1A40A263E26B79
:103D20001340E3631C4AE3681340E36006F046FB7C
:103D30002900300006F056FC8023184A5B00516CC5
:103D400011200B43536407F003FFFD21C720144BE0
:103D5000144A89005A50A36B80003B43A363E36875
:103D6000114A1E43E660E3681D43104BE560195895
:103D70001140802212020A431A50802292051A60D2
:103D80000B4B5F63F8BDC04600F000403CF00040C4
:103D9000FFFFDFFFEFFFEFFFFFFF7FFF0038004077
:103DA0000000FF1F993B0011FF00FFFF00E100E052
:103DB0000000054030B503A804880B20002C0ED16C
:103DC0004968074D08784978090201430A20A94249
:103DD00005D1012120001980024B1B7A137030BDE0
:103DE000192A00008464FF1FF7B5150008AA168879
:103DF0004A680F4F14785278120222430A24BA42BA
:103E000014D10122DBB2019200962A0007F040FC97
:103E1000041E0BD1074B1B68002B07D068782A784B
:103E20000002104342425041013098472000FEBD3D
:103E3000022900000864FF1F30B501250379040042
:103E4000BFB02B4212D00A49408806F08DFF2842AD
:103E50000CD06A46074B69465B8D55801380064B34
:103E600060881B7A1371002204F070F83FB030BDF7
:103E70000064FF1F3043FF1F8464FF1F10B5054916
:103E8000054806F027FF0421044A054806F0E4FE31
:103E900010BDC0460064FF1FFFFF000070BE001190
:103EA0003043FF1F10B5024804F0D2FE10BDC046DB
:103EB000393E0011062310B5837010330371443B63
:103EC00043712A3383714433C371002302220121D9
:103ED00003720E4B027041701C8881724472197A11
:103EE0000273C1729A784273DA7882730322C273C2
:103EF0001A7902745A7942740C2282749A79C274C3
:103F0000DB7903751123C370152010BD8464FF1F76
:103F100010B5122007F084FE104B12220021186009
:103F200007F09EFD002007F053FC012007F0C8FDBC
:103F3000022004F031F9032006F046F9042003F0D2
:103F40006FFB052004F03CF8062001F037FA07204B
:103F500006F062FE082001F01FF810BD0C64FF1F80
:103F600010B507F02DFD012007F05AFD07F050FEB7
:103F7000002010BD094B10B50400984205D001295E
:103F800004D12000064906F0A5FE10BD0229FCD18F
:103F9000013904F01BFE0028F3D0F6E7FEFF000015
:103FA0003264FF1F70B50D7A100004AA2C00168829
:103FB00010221440154220D1002E20D10A78022A66
:103FC00018D14A68517815780E4A0902294391425E
:103FD00005D00D4A914209D01C800A2404E0142225
:103FE0000A491A8007F0CCFD200070BD0C22084958
:103FF0001A80F7E71C800124F6E70824F4E70B2475
:10400000F2E7C046F3FF0000F4FF00008445FF1F05
:1040100048BF001110B504000749084806F05AFED1
:10402000074804F055FD0020E40704D50721054AA0
:10403000054806F011FE10BD3264FF1FFFFF0000AF
:10404000753F0011B0BE00117443FF1F00B50C4B4B
:10405000BFB01A780B4901A800F0ACFC6B4680B2E7
:104060005880002809D06A46074B69461B88138090
:10407000064B0022188803F069FF3FB000BDC04620
:104080001064FF1F1164FF1FCE43FF1FD844FF1FA2
:1040900000B50C4BBFB01A780B4901A801F09CFE8B
:1040A0006B4680B25880002809D06A46074B6946A3
:1040B0005B8D1380064B0022188803F047FF3FB04A
:1040C00000BDC0463A64FF1F3B64FF1F7443FF1FDF
:1040D000D844FF1FF7B50E00377A1C0008AB11005B
:1040E0003D001A8820231D401F423CD13378022B0B
:1040F0003BD173681F785B781B023B431E4FBB426A
:1041000008D01E4FBB4214D01D4DAB4221D00A2512
:104110002800FEBD002A2AD1142C2AD82200F068DB
:1041200007F02EFD174B1C70012CF1D9FFF7B0FFE3
:10413000EEE7002A1BD1202C1BD82200F06807F0E4
:104140001FFD114B04211C70104B187807F0B0FCB8
:10415000DEE7E3B20124009201940A00310007F087
:1041600097FA0500D4E70825D2E70125D0E70B250B
:10417000CEE70D25CCE7C046F3FF0000F4FF0000BA
:10418000022900003A64FF1F1064FF1FBC64FF1F78
:10419000332310B5040003700A220749013007F0E9
:1041A000EFFC064B0F201B681A0AE37222731A0CED
:1041B0001B0E6273A37310BD8464FF1FAC64FF1FEA
:1041C00030B5012503790400BFB02B4213D00B4951
:1041D000408806F0C9FD28420DD06A46084B01A868
:1041E0001B881380FFF7D4FF6B4658800022694676
:1041F000608803F0ABFE3FB030BDC0463264FF1FA5
:10420000CE43FF1F10B5024804F022FD10BDC0468A
:10421000C141001170B5160004AA148805AA1578CA
:104220004A685078117800022A4A08438018052805
:104230004BD807F0FDFA03131E29343F0720032C47
:104240000BD80422121BAA4200D92A0022491A8044
:104250003000091907F094FC002070BD0720112CD4
:10426000FBD81222121BAA4200D92A001B491A802D
:10427000EEE707200E2CF0D80F22121BAA4200D91D
:104280002A0017491A80E3E70720032CE5D8042207
:10429000121BAA4200D92A0012491A80D8E7072027
:1042A000032CDAD80422121BAA4200D92A000E4994
:1042B0001A80CDE70720032CCFD80422121BAA4274
:1042C00000D92A0009491A80C2E700220A201A8070
:1042D000C3E7C046DCD5FFFFFBBE00115864FF1FDB
:1042E000EBBE0011E6BE0011E1BE0011DCBE001104
:1042F00010B50D21024A034806F0AEFC10BDC046C1
:10430000D0BE0011E443FF1FF0B50024274E85B056
:104310003000B47100F0E2F8254D264BEA89297C83
:104320009A422FD10423300003AA00F057F9040069
:10433000300000F011F90123B371002C34D16B4629
:1043400099892B68C9BA4B4329891B4A1B145B18EE
:1043500053806B46D9896B6849BA89B24B436989E6
:104360001B0C5B181548191C1BB2834200DD011C95
:104370000B0400D5002113889180013313802000A5
:1043800005B0F0BD0227220003AB3000009700F01B
:10439000F7F80E230400297C0122300000976B44BB
:1043A00000F0EEF80443C3E71C00E8E7BC44FF1F3D
:1043B0006C64FF1F830500008464FF1F0F2700004B
:1043C00073B5234E300000F089F8224D07236A466A
:1043D0003000297C00F002F904003000002C33D1B9
:1043E0006B461B787F2B2FD800F0B6F86B46D87839
:1043F000F02302041B031A406B469B8816495BBAE4
:104400009BB21A432B68000953432A891B0C9B1843
:104410004B806B465A789B7812031B011A436B68DA
:10442000024353436A891B0C9B180C481A1C1BB28D
:10443000834200DD021C130400D500220B888A8011
:1044400001330B80200076BD00F086F80124F9E7E7
:10445000BC44FF1F6C64FF1F8464FF1F0F27000014
:1044600070B5114C237C002B0FD0382B0ED10F4D83
:10447000280000F033F8CC23AC222800217C9B01DB
:1044800000F0F4F8280000F067F870BD084BE289EE
:104490009A42FAD1054D280000F020F800222800A9
:1044A000217C00F0C5F8EDE76C64FF1FBC44FF1FE2
:1044B0008305000010B5084B1A7C002A09D05B69FF
:1044C000002B06D09847041E01D0FEF799FD20006E
:1044D00010BD0124F9E7C0466C64FF1F70B5C179B7
:1044E00005000C00631E9C411A4BE402E4184900CD
:1044F0000460C9B2007906F0ABF8E979687949003F
:104500000131C9B206F0A4F8E8790930C0B207F069
:1045100067FB0023E36661332360AA795B3B002AD3
:104520000ED022689A43023B134323600A23E361BF
:104530000733236200232363A3630133E36370BD66
:1045400022689A43022313432360462363610633A0
:10455000A361EFE70050004070B500250400036838
:10456000DD66C0790930C0B207F06AF92900207908
:1045700006F00AF82900607906F006F870BD000020
:10458000F8B51E0006AB1D78002304681700E3662B
:10459000616007F0CDFB01238022E3662B002761D9
:1045A0005200013B08D207F0B3FA08200A4A11680A
:1045B000002D03D12800F8BD2261F2E7236F0342EA
:1045C00003D02369013D3370013613685B1A032B56
:1045D000EED90125EEE7C0466008FF1F70B51C004C
:1045E000002305681600EB66696007F0A1FB012354
:1045F0008022EB6623005200013B08D207F088FAC4
:1046000008200A4A1168002C03D1200070BD2A61DD
:10461000F2E72B6F034203D02B69013C3370013664
:1046200013685B1A032BEED90124EEE76008FF1F25
:10463000002370B504681500E366616007F078FB3D
:104640000123E366256107F063FA8020064A8000B3
:104650001168636B034205D113685B1A032BF8D909
:10466000012070BD0020FCE76008FF1F70B51D0031
:10467000002304681600E366616007F059FB01231C
:10468000E36626610F33626B1A42FCD02B0A23616A
:104690001023626B1A42FCD0EDB2256107F038FAA4
:1046A0008020074A80001168636B034205D11368BC
:1046B0005B1A032BF8D9012070BD0020FCE7C0462F
:1046C0006008FF1F70B51E00002305681400EB662C
:1046D000696007F02DFB0123A619EB660F33B44286
:1046E0000ED107F015FA80200A4A800011686B6B22
:1046F00003420CD113685B1A032BF8D9012070BD5B
:1047000021782961696B1942FCD00134E7E7002068
:10471000F5E7C0466008FF1F10B5084CE368002BA2
:1047200008D1074B1B685B045B0C0A336360054BC5
:104730001B68236007F08CF8A06010BDAC64FF1FFD
:10474000C8F00040CCF0004010B507F0F1FA0F4B74
:10475000996A9A6A8A42FBD10D4C6268A0688A18ED
:10476000121A531E884200D31300A1602168DA0B8D
:1047700052185B0407495B0C636022600B60064BB8
:104780001A6007F0C5F9206810BDC04600F000406F
:10479000AC64FF1FC8F00040CCF0004070B51F4C67
:1047A00023793F2B01D93F2323711D4B22791A70A6
:1047B0001878C0B207F094F918231A491A4A0B80E6
:1047C0001A4913800B805380A379194980200B80EC
:1047D0000C21938001334B43164D191C0001834279
:1047E00000D9011C2980D1806379002B11D10133BC
:1047F0006371237A012B01D8022323726279237A11
:104800000D4853430A21584307F03AF80B4D2860EE
:1048100070BDA02BEDD9A023EAE7C046A064FF1F1E
:10482000480AFF1FD644FF1FAC46FF1FD444FF1F9A
:10483000D244FF1FD044FF1F710200009064FF1F8D
:10484000F8B513210020FEF7C9FD114C011E114DD2
:1048500009D10C22104BC1CBC1C4280007F000F9CC
:10486000FFF79CFFF8BD0C2220000C49FEF78AFDE3
:104870000C2802D0084B43CB43C40C222800084923
:10488000FEF780FD0C28EBD00C220021E5E7C046A6
:10489000A064FF1F6C64FF1F3CBF0011FC0C0000F4
:1048A000F50C0000F0B51D4C8022A54404008820C2
:1048B00069465201400507F01BF8902212016A4434
:1048C0001300200032C832C316C816C38023144C0C
:1048D000144FA6689B033343A3603B6007F018F8AE
:1048E0008823A0685B05C01806F09AFF002588237E
:1048F00029008022A0685B05C01840196944520055
:1049000007F0F6F880230135FF355B019D42EED1BB
:10491000A6603E60044B9D44F0BDC046FCEFFFFF27
:104920001C46FF1F9808FF1F04100000F0B504008C
:1049300087B0002825D0684607F0FAF81B4C0228FB
:1049400006D106226946200007F0D2F9002816D0C9
:104950006946002301250F262F00E25C0133100970
:104960001030874038002F00324097403A00024311
:104970004A610439062BEFD16846FFF793FF07B071
:10498000F0BD182269460A4806F0B2FF6A46A30045
:10499000D358013305D01822FF21684607F060F88C
:1049A000EAE70134062CF1D1E9E7C0466509FF1FAB
:1049B00000090011F0B5002504000E0085B0AA42E0
:1049C00000D186E04B1C087801934B7889783779C1
:1049D00009021943F3783F061B040B431F43039757
:1049E00020706570252800D196E033D8112813D89F
:1049F00006F0FEFF69002501250125012501AA0019
:104A0000B800B10025012501250125012501250159
:104A100025012501FF001F01232800D1D8E0DB2854
:104A200000D02EE1042A00D8ACE01025052A05D0DC
:104A3000551F2A003800711D07F0A2F80522310029
:104A4000200007F09DF82A003900601D07F098F853
:104A500005353EE0562859D010D8332800D19DE0C6
:104A6000552839D02628DAD19C4B2900132218006A
:104A70001D0006F0F5FFFEF7C3FA5CE0712800D1D7
:104A800077E0722800D180E0602800D18BE0DC283C
:104A9000C5D1022A00D875E07378BFB26370B378CD
:104AA000A370032A05D0033A390092B2F01CFEF736
:104AB000A3FB10223900E01CFEF764FCC51C002893
:104AC00007DA60705CE00C222000854907F058F896
:104AD0000C25280005B0F0BD013A824D0C2A13D8F0
:104AE000002A0AD02800019907F04AF8FFF756FE7D
:104AF0000C2228007C49FEF77FFB29000C22601C59
:104B000007F03EF80D25E4E70C22EBE7754D774BF7
:104B10002A0043CB43C2E9E7013A704D0C2A11D871
:104B2000002A08D00199280007F02AF80C22280052
:104B30006F49FEF761FB29001322601C07F020F883
:104B40001425C6E70C22EDE705226A49601C07F030
:104B500017F80625BDE712226749601C07F010F818
:104B60001325B6E708226549601C07F009F80925F6
:104B7000AFE77178F72905D8614B188801F088FDF7
:104B80000225A6E7FF236370FAE75E4B012A03D0F4
:104B900072785A706270F3E75B78F4E72000FFF7F1
:104BA000F7FA050095E7013A574D072A0ED8002A73
:104BB00005D00199280006F0E3FF01F047F829002D
:104BC0000722601C06F0DCFF082582E70722F0E7D9
:104BD000042A04D94D4D2F6006F03AFEA860FFF775
:104BE000B3FD0422039003A9601C06F0C9FF05254C
:104BF0006FE7474D062A15D906222800019907F0CC
:104C000077F800280ED006220199280006F0B8FF98
:104C1000062240492800FEF7EFFA0123394A51786D
:104C20000B43537029000622601C06F0A9FF0725DC
:104C30004FE7012AA6D07078FFF778FEA0E7012899
:104C400000D0ECE6931E344F1A2B04D87378002B57
:104C500009D100F015F9314B39001D78601C6A1E2E
:104C600006F08EFF35E7551E2A000199380006F040
:104C700087FF2B49AAB23800FEF7BEFA00F036F9DA
:104C8000E9E7DA281DD1042A00D87BE7082A15D9DC
:104C9000B37972791B021343F27912041A43337AFF
:104CA0001B0613433B603B68052231002000039341
:104CB00006F066FF0422601D03A956E7FE23637019
:104CC000F1E7DE2800D05DE7511E012A01D1002561
:104CD000FFE6019800F0A0FFF9E7C0466C64FF1FF3
:104CE00048BF0011A064FF1FFC0C00003CBF001176
:104CF000F50C00007864FF1F5864FF1F2046FF1F5B
:104D0000D844FF1F9C64FF1F7545FF1FAC64FF1F45
:104D10006509FF1FADAC00009D66FF1F9B66FF1F6E
:104D2000AEDE000070477047020010B5094B0A3232
:104D3000094C92B2DA815A8298811882207802F066
:104D40000DFB0422054B012120781A7006F0B0FEFD
:104D500010BDC046AA45FF1FE666FF1FE566FF1FA0
:104D6000013870B5042809D806F062FD0309280847
:104D70001200234B0221187806F09AFE70BD204BDA
:104D80000821187806F03CFF00221E4B1A72F5E746
:104D9000802200241B4B1A4D52001A8108211A68E8
:104DA0002878DC7207F01CF82100287806F020FD36
:104DB000012000F051FE00F049FFDFE7104B082111
:104DC000187806F01DFF1048FFF774F80F4B104AD3
:104DD0009B79002093800F4A13808022094B520058
:104DE000D8721A8100F038FE00F030FF0A4B5B7871
:104DF000002BC3D0094A136006F05AFDBEE7C04637
:104E0000BC64FF1F9064FF1FE144FF1FA064FF1FED
:104E1000AC46FF1FD244FF1F9C64FF1F34F00040CC
:104E200010B501290BD1012809D1054B1B78002BA6
:104E300005D02622034B04485A72FFF775FF10BDB8
:104E4000BE66FF1F9064FF1FC40900000300F0B599
:104E50000A4D8E18B14202D152008018F0BD0C7874
:104E60002F6824093C5D0F271C700C7801313C40F1
:104E70002F683C5D5C700233ECE7C046CC44FF1FFA
:104E80000D22114B10B51A700C23104C10492370D1
:104E9000093A033B0F48637006F072FE2D2301228E
:104EA0000D490E48A371FFF7D1FF01220C49FFF70E
:104EB000CDFF01220B49FFF7C9FF00220A4910006C
:104EC000FEF79AF910BDC046BA66FF1F9B66FF1F2A
:104ED000FBBE00119D66FF1F6709FF1FA266FF1F33
:104EE0006609FF1F6509FF1FAEDE000070B5124C9A
:104EF000132220001149FEF745FA114D002817DD55
:104F0000AB78002B14D0431C2B7009236B7000234B
:104F100000190370287829000130C0B206F078FC2F
:104F2000297822000139C9B2002005F0B3FD70BD17
:104F3000FFF7A6FFEEE7C0469D66FF1FAEDE00004E
:104F40009B66FF1F10B5114B1A781870002A0ED0FF
:104F500000280BD10E4B1A78062A07D85423D340C9
:104F6000DB0703D50B4B187802F0F8F910BD0028C9
:104F7000FCD0074B1B78012B02D0033B022BF5D84A
:104F8000044B0121187806F093FDEFE7BE66FF1F82
:104F9000E566FF1FE666FF1F70B54A4E4A4A4B4959
:104FA0003070012005F002FC00F0B4FEFEF728F896
:104FB00006F01EFE032246494648FFF747FF2D2410
:104FC000030004221C7044490130FFF73FFF3023E7
:104FD0000470424D424C437083702E3B06222000E9
:104FE0004049EB87FEF7CEF9062813D0200006F0E3
:104FF0009FFD022809D00321200006F099FC8D2393
:10500000E3706E3B2371193363710622200035492A
:10501000FEF7F2F8344B1B68FC335C64FFF766FF65
:105020000020FFF78FFF314C314A0121314B1278BC
:10503000207802F055F9304A304B12780021207860
:1050400002F04EF901222E4B1A702E4B9B78552BF5
:1050500031D12D4B3B325A722C4B2D4AAB81EA8118
:105060002B826A822021307806F0CAFE012040425D
:1050700005F05CFD0120404205F0F8FDFFF738F92E
:10508000FEF7FCFE00F0A6FC01204042FEF7C2FF46
:10509000012006F0EDFCF72001F0DEFA0121307866
:1050A00006F006FD307802F0B5FA1A4806F0F0FC7A
:1050B000FEF7F2FD70BD6422174B5B7953431A0073
:1050C0000A32CBE7BC64FF1F254D0011214E0011B1
:1050D0002046FF1F5864FF1F7864FF1FAA45FF1F6B
:1050E0006509FF1FADAC00004467FF1FE666FF1FA8
:1050F0000045FF1FE144FF1FBA66FF1F9B66FF1FAD
:105100008C66FF1F9C64FF1F9064FF1FC409000092
:10511000CE090000BE64FF1FA064FF1FF8B50A009F
:1051200020230D001A40194257D0574B1B78002BF3
:1051300050D0FFF709FB554B554C564E99686268A5
:10514000737A8A1ADB039A4202D36160FEF7A4FDE8
:10515000327A217A531EDBB2994205D1FFF780F9EA
:10516000002000F0A9FD0FE09142F9D30023237243
:10517000FFF7A0F9012000F09FFD474F3800FEF730
:1051800099FE390006F0ECFB637A002B1FD0013B3F
:10519000DBB26372002B1AD1404B9B78552B01D1A7
:1051A00006F086FBE37A002B0CD000233C4A3A4FF2
:1051B000E3721388380001331380FEF77BFE390059
:1051C00006F0CEFB642370795843FFF7ADFD237AD8
:1051D0000133237220206840F8BD0BB2002B0ADA9D
:1051E000304B187806F08CFD002801D006F040FD09
:1051F00080200002EFE70224214206D0244B012048
:105200001A72FFF79FFE2000E5E70B071ED5FFF798
:105210009BFA1E4B1E491F4C98684A68637A821A93
:10522000DB039A4202D34860FEF736FDFFF742F9EE
:10523000FFF716F9012000F03FFD00F0E5FB2368C1
:10524000DB0701D5FEF7DEFF0820C4E7102421426A
:1052500006D00D4B1B78002BD5D1FEF723FED2E7ED
:105260000124214207D0104800F06CF806F0E0FC61
:1052700000F008FDC7E70424080020402142ABD01D
:10528000FEF7E4FEBFE7C046BE66FF1FAC64FF1F2B
:105290009064FF1FA064FF1FE144FF1F9C64FF1F79
:1052A0008464FF1FBC64FF1FC444FF1FF0B51B4B89
:1052B0001B4F1B883A8804001A4E1B4D85B09A423A
:1052C0000DD832889A420AD3184B1A882B889A42F2
:1052D00005D1174A174B12881B889A421BD005200C
:1052E00001F010FA3B8802AA1380338801905380A2
:1052F0002B88114D93800F4B02A91B88D3800F4B35
:105300002A78188802F02CFF0D4B08212878019A82
:105310001C7006F075FB05B0F0BDC0468A66FF1F25
:10532000D644FF1FD444FF1FD244FF1F8866FF1FCF
:105330008666FF1FD044FF1FE666FF1FD844FF1F8D
:105340008466FF1F13B50C4B1C78002C11D100286C
:1053500001D00A4B18600A4A0A4B11780A4A1078A1
:105360000A4A01920A4A0092002205F08BFA2000B4
:1053700016BD1124FBE7C046E566FF1F8066FF1FD0
:10538000E466FF1FD466FF1FE666FF1FC066FF1FAF
:10539000C466FF1F10B5064B12201B78052B06D1E3
:1053A000044B13221988044B187801F087FB10BDB9
:1053B000E566FF1FD844FF1FE666FF1F10B50024F7
:1053C0000122114B52421870104B1C70104B1A8066
:1053D00002F020F904220F4B21001A700E480C3203
:1053E00006F0FEFA102221000C4806F0F9FA072216
:1053F0000B4B1C600B4B1C700B4B1C700B4B1A7037
:105400000B4B1C7010BDC046E666FF1FE566FF1F14
:10541000D844FF1FE466FF1FD466FF1FC466FF1F4A
:10542000C066FF1F9A66FF1F9966FF1FDA44FF1FC1
:105430009866FF1FF8B5174C0600257806A81424B7
:105440000078052D23D1B41F134FA5B21824BD42F7
:105450001DD88D1FADB2BD4219D8FA256D00AA42E4
:1054600015D21D000D4F0A3DADB2BD420FD80C4CF8
:1054700026800C4C21800C4900240A800B4A1380A2
:10548000FFF714FF0A4B0421187806F0B9FB20003F
:10549000F8BDC046E566FF1F790C0000750C0000E2
:1054A000D644FF1FD444FF1FD244FF1FD044FF1F28
:1054B000E666FF1FF0B50BB20D0089B0002B00DBD4
:1054C00070E1A44E307806F01BFC041E50D0037827
:1054D000A22B00D122E1D02B1AD0912B45D14378B9
:1054E0000E2B42D19C4B82889A423ED19B4A8368C4
:1054F0001278052A39D1032018567F2835D0984BC9
:105500001B68002B31D05B68002B2ED098472CE015
:105510008078072829D806F08BF90428183F3F74B3
:10552000A8D86378002B0CD101218C4B19708D4BBE
:105530001A78002A5BD08C4B307801F0D1FE00281D
:1055400055D00722854B1A7051E061780029F8D1B7
:10555000E378002B11D0854A854B1278307801F022
:10556000BFFE60706378002BEBD1200006F080FB5B
:1055700080200002684009B0F0BD784B1B78022BF8
:10558000F3D00121307806F07BFA0028EAD101211E
:10559000307806F08DFAE5E76378002BD1D16F4FB4
:1055A000032807D13B78052B02D101333B701EE065
:1055B0000223FBE76F4B1A886F4B0293002A0BD034
:1055C0001B78002B03D00121307806F019FA3B78C4
:1055D000062B04D1013BE9E7029B1A70F7E7042B85
:1055E00041D10121029B3078197006F061FA5C4BC1
:1055F0001B68002BB9D01B68002BB6D0574A107817
:1056000084E76378554F002B27D10622211D5B4884
:1056100006F0B6FA62895A4B5A491A80A2895A4B47
:105620001A80E3890B800521397058490A80584A4D
:105630001380228A574B1A80574B1B78012B09D1B4
:105640001F2001F05FF8FA229200424304213078D3
:1056500006F0D6F90022484B75E7312B00D070E7F1
:105660000022454B1A700323A0E70622002143487D
:1056700006F0B6F90023454A04211380444A3078E5
:105680001380444A138006F0BBFA0821307806F0F4
:10569000B7FAA379083B5A425341304A0333137097
:1056A000304B1B78002B06D0334B30781A78002A09
:1056B00006D001F053FE0122314B52421A8096E788
:1056C0000121197006F0F4F9F5E70821307806F0A9
:1056D00097FA6378002B00D047E72C4B2D4F0293AD
:1056E000E388029A04211380294B3078039323899D
:1056F000039A138063893B8006F0C2F9002800D02A
:1057000033E7264B1B68002B00D12EE70399029844
:105710003A88098800881B68984726E74379132B45
:1057200000D022E70389012B0AD11D4B1B78022BE5
:1057300006D10821307806F063FAFFF72BFE14E754
:10574000052000F0DFFF08210200307806F058F94C
:105750000BE7C046E666FF1F05140000E566FF1F65
:105760008066FF1F0045FF1FE144FF1FBA66FF1F51
:105770009B66FF1FBC66FF1FBE66FF1F8D66FF1F77
:10578000D844FF1F9466FF1F9666FF1F8A66FF1F9F
:105790008866FF1F8666FF1F8C66FF1F7C66FF1FE3
:1057A0008466FF1F8020C001014200D0E2E6CB07E3
:1057B00031D5324B1B78002B1DD0314E05AC3378E0
:1057C000052B1AD1023B23702E4B21001B7823722C
:1057D0002D4B1B7863722D4B187801F025FD0028A6
:1057E00009D007202A4B30701B68002B03D01B68A0
:1057F000002B00D098470120BCE60E20254B062246
:105800001B7825492370254B1B78637002ABC018A9
:1058100006F0B6F9D8E7022308001840194209D06B
:10582000174B1B78052B03D11D4B188806F018F871
:1058300002209FE60424214203D0FFF737FD200019
:1058400098E6082308001840194200D193E6154B4A
:105850001C78012C03D0022C0DD008208AE6124BB4
:10586000124A134913481B8812880988008800943B
:10587000FFF7E0FDF1E7FFF78DFDEEE7BE66FF1FE6
:10588000E566FF1FDA44FF1F9866FF1FE666FF1FED
:105890008066FF1F9A66FF1FDB44FF1F9966FF1F8C
:1058A000D844FF1F8466FF1FD044FF1FD244FF1F50
:1058B000D444FF1FD644FF1F10B502A804880B2054
:1058C000002C10D1496808784978090201430C4836
:1058D000814209D1022119800A4B59881170DB7865
:1058E00000205BB2537010BD074C0A20A142FAD1D0
:1058F00002211980034B998811705B79F0E7C0464B
:105900006E2A00008464FF1F6F2A0000F7B515009F
:1059100008AA16884A680F4F147852781202224358
:105920000A24BA4214D10122DBB2019200962A0065
:1059300005F0AEFE041E0BD1074B1B68002B07D0F1
:1059400068782A780002104342425041013098475B
:105950002000FEBD02290000F866FF1F30B50125BA
:1059600003790400BFB02B4227D01549408805F0C9
:10597000FBF928420DD06A46124B69465B8D1380B5
:1059800002235380104B5B8893806088002202F0D2
:10599000DDFA0E49608805F0E7F9C0070DD56A46C3
:1059A0000B4B69461B88138002235380064B9B8850
:1059B00093806088002202F0C9FA3FB030BDC04633
:1059C000F066FF1F0445FF1F8464FF1FE866FF1F8A
:1059D0005E45FF1F10B5074C0749200005F07AF916
:1059E0002000064905F076F90721054A054805F02B
:1059F00033F910BDFFFF0000F066FF1FE866FF1FD0
:105A0000C8BF00110445FF1F10B5024803F020F97C
:105A100010BDC0465D5900110221430888400B406B
:105A20000A31084003430E20024AD17881430B43D8
:105A3000D37070477545FF1F064A1379410705D596
:105A400080210B4380011371907170477F210B40BF
:105A5000F8E7C0467545FF1F054A5378002803D074
:105A600080210B43537070477F210B40FAE7C046FB
:105A70007545FF1F0F21114BDA780A40DA70502864
:105A800010D901310A43DA702022D9780A43DA703A
:105A90004022D9780A43DA708022D97852420A43E8
:105AA000DA7005E03C28EFD82828F1D81428F3D87C
:105AB0000122D9780A43DA707047C0467545FF1F46
:105AC000F8B57F23324D04006E789E43314B9842E7
:105AD00005DD76232B70363B33436B70F8BD2E4BC0
:105AE000984203DA58232B701433F5E783B21A0077
:105AF00000215F32294892B2294F297082422DD964
:105B0000A9708C4203DA5B421CB220232B7005344F
:105B100020B20A2105F0B4FE04B2FA239B009C4295
:105B200033DB80232A785B4213432B7064212000EF
:105B300005F0A6FE0A2100B206F082F809B22A7822
:105B40007B5C13432B700A21200005F099FE0A218B
:105B500000B206F075F809B27B5C0AE08022AA70F8
:105B6000002CDADA5B421CB220232B705F23092C55
:105B7000E9DC1E430A2120006E7006F061F809B2CC
:105B8000AA787B5C1343AB70A8E7632CCEDCEDE70F
:105B90007545FF1F1B4E00001DFCFFFF2A0800007B
:105BA000F2BF00117F23F7B5194FCD013E790400F4
:105BB0009E433E71EDB2632806DD093B33433B71E2
:105BC00040231D437D71F7BD0300093304DA5823D8
:105BD00033433B716C23F4E70E4B019300280BDA3F
:105BE0000423444224B23B710A21200006F028F825
:105BF000019B09B25B5CE4E70928F5DD0A2105F0A9
:105C00003FFE019B00B21B5C1E433E71ECE7C046A9
:105C10007545FF1FF2BF0011F8B50A4F05003B782C
:105C20000E00002B0CD0084C2000FEF757FC330070
:105C30002A0020003978FEF745FD2000FEF78CFC95
:105C4000F8BDC0460467FF1F7C45FF1F70B50A4EB4
:105C50000A4D07223100280006F04AF8002809D032
:105C6000074C31000722280005F08AFF0821200098
:105C7000FFF7D2FF70BDC0467545FF1FFD66FF1FD1
:105C8000FC66FF1F7F2210B50A4B59789143033AF7
:105C90001A70103A0A435A7078220E219A70DA78F4
:105CA0008A43DA7006221A7129325A71FFF7CEFF41
:105CB00010BDC0467545FF1F10B5002824D0134CF9
:105CC0000A210223E05E05F0DBFD00B2FFF7F8FEDB
:105CD0000423E05E642105F0D3FD012100B2FFF74B
:105CE00061FF207AFFF7C6FE0320FFF795FE002034
:105CF000FFF7A2FE064B1878053843425841C0B260
:105D0000FFF7AAFEFFF7A2FF10BDC0468464FF1F85
:105D1000E566FF1F70B50024094D2800AC71FEF741
:105D2000DDFB10233E212800064AFEF7CBFCA042F3
:105D300000D13E34044B28001C70FEF70DFC70BDF2
:105D40007C45FF1FE2BF00110467FF1F0200F0B592
:105D500001270A480A4E51188B1A002B00DCF0BDAF
:105D6000082415784308684038404000805B013CB7
:105D700058406D08002CF5D10132EDE7FFFF00001F
:105D800002C00011F0B500250F269D4200DBF0BDDA
:105D90004C5D070944403440A400A05801357840C8
:105DA000F3E70000F0B589B06A460D000B000F273D
:105DB000110010351C780133260024093E4016706E
:105DC00054700232AB42F5D12023024AFFF7DAFFCA
:105DD00009B0F0BD08C00011F0B54E780B7889B05D
:105DE00036020C00170001901E43012A61D9954B21
:105DF0009E4200D877E001339E421CD1062A17D17B
:105E0000CA788B7812021A430B791B0413434A7920
:105E100012061A438C4B5A6100221A705A808B4A20
:105E20005A608B4A9A608B4ADA60002009B0F0BD54
:105E300088225205EEE7884B9E423CD182498B78FE
:105E4000002B00D0F6E00C2A31D10F22A378934327
:105E5000E278120213432279120413436279120684
:105E600013434B60E279A07912020243207A0004C6
:105E70001043627A12060243CA60E27AA07A1202E2
:105E8000024376484A81834208D804236E4914228B
:105E900001980B7005F074FE1420C7E71201D218A8
:105EA00089235B059A42F0D801238B70BDE7022A53
:105EB000FAD00523EAE76A4A01239642E6D1FFF7C2
:105EC00069FA052F0CD9E378A2781B0213432279D3
:105ED00012041A4363791B061343624A0393136047
:105EE00005F0E6FCA1E7584D2B78002B9DD1AB784F
:105EF000002B00D1A0E02B8901339BB20093B34269
:105F000000D091E0132AD4D9CF7C8B7C3F021221A0
:105F100020001F43FFF71AFF874200D08EE0002EBB
:105F20003DD1E378A2781B0213432279E968120479
:105F30001A4363791B06134303930A228B4212D13F
:105F4000FF23A370E370237163716B89002B09D168
:105F5000E37B227C1B0212041343A27B13431B0925
:105F600001336B8100226B89002B8ED0002A67D110
:105F7000686837013818000B6B690003039098427A
:105F800005D9686105F04CFCEB780133EB7068686B
:105F90001022A11C381805F0ABFD2E8145E76F8952
:105FA000009A7B1E9BB293423AD1E278A378120208
:105FB0001A43237905A81B04134362796C681206FF
:105FC0001A43EB6800920392211D0C22049305F002
:105FD000D7FD0120260004A940421036FFF7E2FE5B
:105FE000013F012F17D1009A0B232861824200D074
:105FF0004CE704221C49200005F07AFD042203A985
:10600000686805F075FCE968039AFF23914200D1A6
:106010003CE7F73B3AE73100FFF7C4FE1036DFE715
:106020000923B742A4D831E7009BB34200D9FCE66C
:1060300007232BE7022329E7032327E7062325E786
:106040000A2323E7FFFE00008445FF1F0000011123
:10605000FFFF00005048593601FF0000FFFF00110C
:1060600002FF000034F000409045FF1F10B5034CC4
:106070000B000122210000F06BFA10BD2D6200110F
:106080000B8870B506000D000224162B11D92B00C9
:106090000322094900F05CFA041E0AD1074B2A8842
:1060A0001B88191C934200D9111C300089B200F0E2
:1060B000EFFA200070BDC046596200115E67FF1FF5
:1060C00010B54A780400013A0B000220012A07D8D3
:1060D0000A78002A04D005222000024900F038FA8C
:1060E00010BDC046876200110A7810B50B0004008D
:1060F0000220002A04D007222000024900F028FADA
:1061000010BDC046336300110A7810B50B000400BF
:106110000220002A04D009222000024900F018FAC7
:1061200010BDC0469963001110B5034C0B000B2243
:10613000210000F00DFA10BDC963001110B5034C29
:106140000B000D22210000F003FA10BD3B6400118A
:1061500010B5034C0B000F22210000F0F9F910BD1F
:10616000956400110A7810B50B0004000220002A83
:1061700004D011222000024900F0EAF910BDC04607
:10618000A5640011002310B51322190000F0E0F9F6
:1061900010BD000010B5034C0B001722210000F0C9
:1061A000D7F910BDF7640011002310B519221900AA
:1061B00000F0CEF910BD000010B5034C0B001B22FF
:1061C000210000F0C5F910BD31650011F7B58489D3
:1061D0000D0006000121002C22D000238268D35636
:1061E0001778002B1EDA0C2C1AD90C3CA4B2131908
:1061F00040880093230002F086FE431E9841013040
:106200007B06DB0F6B703F23013C1F40A4B228705C
:10621000AF70AC80002C07D0B3680133AB600021B5
:106220000800FEBD0020EBE7AC60F8E70B780370D8
:106230004B8843704B881B0A83700B79C370042012
:1062400070470420022B06D10020537811781B02DE
:10625000009A0B43138070470B8803700B881B0A4E
:106260004370022070470420009983420AD153787A
:1062700010781B0203430B80D37890781B020343F2
:1062800000204B807047F8B50D004B7801240021A9
:10629000461C03702B788B4201D82000F8BD6B7828
:1062A000B01C4F1C012B10D1890069184B880222A9
:1062B00033704B88B9001B0A7370691805F030FD04
:1062C00004360434A4B2F9B2E4E7122359436B183C
:1062D0005A88043132705B8810221B0A7370691867
:1062E00005F01EFD12361234ECE770B5049D140063
:1062F0001E00052B01D8042070BD637812781B02A4
:1063000013432B80E378A2781B02134302226B8095
:106310002A71211D681D063E05F002FDB2B22A81D8
:10632000F02AE8D82800A11D0A3005F0F9FC002069
:10633000E2E7002310B50A789A4201D8900010BD18
:106340009A008A185488013304705488DBB2240AF6
:106350004470948884709288120AC2700430EAE70C
:1063600010B51100029C062B04D004201022142B1F
:1063700001D010BD022222714B7808781B02034322
:106380002380CB7888781B02034363800431601D2F
:1063900005F0C6FC0020ECE710B50C788B780431D2
:1063A0005C43E4B203702200013005F0B9FC601CCC
:1063B00010BD0420022B06D10020537811781B0257
:1063C000009A0B431380704710B50C000A88023105
:1063D00005F0A6FC208810BD70B504000D000498DF
:1063E0001100012B01D8042070BD167852781202DA
:1063F000324302800200F83255701470E825002CF8
:1064000000D10C35023B9AB24280AA42EBD802314D
:10641000043005F085FC0020E6E704200099834263
:106420000AD1537810781B0203430B80D3789078FD
:106430001B02034300204B80704710B50C000A88F4
:10644000023105F06DFC208810BD000070B50121FF
:106450001E000420049C0E400B4218D1CB40DDB23C
:106460008D4214D90A49DBB2098899420FD323001F
:10647000F6331D703300580011184978165C090274
:10648000314301332152D9B28D42F4D8002070BD7E
:10649000A445FF1F10B50C000A88023105F040FC2E
:1064A000208810BD10B50C788B7804315C43E4B2C1
:1064B00003702200013005F033FC601C10BD10B5E4
:1064C00011000298032B01D8042010BD14785278D3
:1064D000043B120222430280CA788C7812022243C3
:1064E00042809AB28280F22AEED80431063005F05A
:1064F00017FC0020E9E710B50C000B8803700B882F
:106500001B0A43704B8883704B881B0AC3708A88B0
:106510000430063105F004FCA088043080B210BDC0
:106520000420012B03D100201378009A13707047C8
:1065300010B50C000B8803700B881B0A43704A8847
:106540000230043105F0ECFB6088023080B210BDEF
:10655000F0B589B003931E4B029242000700D05A57
:10656000019102F020F81325061E2DD0029B012474
:106570000370019B002B04D0001903999847001960
:1065800084B26B461B7A5BB2002B0FDA1021380005
:1065900002F01CFB1925002813D130003219E1B29A
:1065A00002F066FC051E0CD10C34A4B2042304AA2C
:1065B000380005A993800696948101F0AFFD051E71
:1065C00002D0300005F06CFB280009B0F0BDC046D9
:1065D0005C67FF1F70B505000C0000280CD0002080
:1065E000814209D010222000044905F099FB0120C6
:1065F0002B7823736B78637370BDC04648C000115D
:10660000F0B506000D0017001C0085B002291BD054
:106610000020102907D1022B07D0102B03D115E041
:106620000020102C08D005B0F0BD69463800FFF7F7
:10663000D1FF2A0069460BE069463000FFF7CAFF28
:1066400022006946380004E0022BE9D12A00390013
:10665000300005F03DFAE6E7031CF72800D9F723E0
:10666000032008499AB2013A0B80D3170340064928
:106670009B189B100B80D30F04499B185B100B8059
:106680007047C046A845FF1FA645FF1FA445FF1F32
:10669000034B1B888B4202D3024B4000C152704710
:1066A000A845FF1F5C67FF1F014B4000185A704749
:1066B0005C67FF1F1722014B1A8070475C67FF1F42
:1066C00070B505000E2005F00BFB041E13D0D0237F
:1066D000037000230622837007494570033005F0DC
:1066E0001FFB064B2100DA8A62811B7E2373044B59
:1066F000187805F04DFB70BD7867FF1F6867FF1FB6
:10670000F845FF1F262803D8024B4000C05A7047A7
:106710000148FCE7AA45FF1FFFFF000070B5060017
:106720000C00094D1C220021280005F059F9074BE7
:106730001E70074B1C7005F06BFB0123002801D075
:10674000002312202B7070BD6867FF1FF845FF1FE4
:106750008967FF1F70B505000D4C0800E260A1605D
:1067600010220021656005F0CBF9012803D110212A
:10677000A06802F058FD10220021280005F0C0F9A1
:10678000012803D11021606802F04DFD70BDC046A4
:106790006867FF1F70B5041E05D1002903D00622CB
:1067A0000D4805F0BDFA0D4B1D78012D11D1002CBF
:1067B00005D102221A7005F0B3F9280070BD00223D
:1067C0001A70074B1B78FF2BF7D02000FFF778FFDC
:1067D000F3E70025F1E7C0467867FF1F6867FF1FF2
:1067E000F845FF1F030010B5002801D1002010BD9F
:1067F00000780B4A002803D15988D1821B7913767F
:106800001378022BF2D10023984200D10333137086
:10681000044B1B78FF2B01D0FFF752FF0120E6E766
:106820006867FF1FF845FF1F002911D000280CD012
:106830004B79012803D140225242134303E03F2207
:106840001340032802D001204B7170474022F4E727
:106850000800FAE770B5094D0100287800280BD030
:10686000074C0622200005F05BFA21002878FFF78C
:10687000DBFF200005F0E4F870BDC0468867FF1F0D
:106880006267FF1F00290AD0012808D13F224B79F7
:106890009343C02B03D0403B5A425341981C70474E
:1068A00070B5174D06002B78FF2B15D00A2005F088
:1068B00017FA041E10D0D0230370C83B8370114B0D
:1068C00011491B784670C3700622043005F028FA7F
:1068D0002100287805F05CFA0C4B1B78012B0DD1B8
:1068E0000B4B1B68002B03D09B68002B00D09847F4
:1068F000084B04211878084A05F072FA70BDC046AA
:10690000F845FF1F8867FF1F6267FF1F8467FF1F2F
:10691000B067FF1FB467FF1F60EA0000014B986873
:106920007047C0466867FF1F014BDB6818687047F7
:106930006867FF1F074B10B5DA68136801331360EF
:10694000054B1878FF2803D08021C90105F0B0F865
:1069500010BDC0466867FF1FF845FF1FF7B50E0062
:1069600002F0C8F8051E1CD00E4B06621F78002FDF
:1069700000D10778AB791020019305F0B1F9041E1E
:106980000FD0D0230380C73B8370019BE91DC370E8
:106990000622043005F0C4F921003800E66005F055
:1069A000F7F9F7BDF645FF1F014B18787047C04651
:1069B0008867FF1F054B002805D1054B1A78054B4A
:1069C000002A00D1014B18007047C0467867FF1FAE
:1069D0008867FF1F6267FF1F014B58687047C046FA
:1069E0006867FF1F024B1868431E9841C0B270478A
:1069F0008C67FF1F421E03000120152A03D9FF3BAD
:106A00005A425341D8B27047F0B51C0000230E0023
:106A100085B0039002920B70029A934201D300203A
:106A200019E0E55C5A1CD2B2002DF8D00298511939
:106A30008142F4DC0233DFB2A35C18000193FFF75C
:106A4000D9FF002807D0013D019A0399EBB23370BA
:106A50008A4202D1E01905B0F0BDDB19DBB2DBE7F9
:106A600010B50C0002F09EF803001220002B03D09A
:106A70002100588804F08CFF10BD000070B50E4D49
:106A800084006359002B15D0186A002801D005F046
:106A90001FF92B59586A002801D005F019F92B5914
:106AA000986A002801D005F013F9285905F010F96B
:106AB00000232B5170BDC0469867FF1F1C4B70B55B
:106AC00004000E00150099420AD11A4B1B68002BD6
:106AD00001D1122070BD1B68002BFAD09847F9E74E
:106AE000154B994215D1134B1B68002B0AD01B681C
:106AF000002B07D09847002804D1104B1C70104B76
:106B00001D70E7E729002000FFF7AAFF0028E1D168
:106B1000F3E7080001F0EEFF0028DAD00378032045
:106B2000A342D7D12900300004F032FFD2E7C0469B
:106B3000FEFF00009467FF1FFFFF00009167FF1F2B
:106B40009067FF1FF7B50400808801F0D3FF002590
:106B5000A84203D00578A08802F008F81C4E3378CC
:106B6000002B1FD0AB421DD11A4B28001978FFF71C
:106B700077FF002818D000233370A3790820A77866
:106B8000A688019305F0ACF8011E0DD0D023037048
:106B9000CA3B8370019B477086808371280005F093
:106BA000F7F801E0002DE8D1A0880B4B8200D35804
:106BB000002B01D0FFF762FF1721A088FFF768FDC7
:106BC000A08801F027FDA08801F0FEFDF7BDC046BA
:106BD0009167FF1F9067FF1F9867FF1FF0B587B091
:106BE0001D000CAB1B88070001930DAB1B88142004
:106BF00002930EAB1B88160003930FAB1B8800910A
:106C0000049310AB1B88059305F06AF8041E1AD094
:106C1000D0230370CB3B47708370C67006222900D7
:106C20000430002D11D005F07BF8019B2100638119
:106C3000029B0098A381039BE381049B2382059B15
:106C4000A37405F0A5F807B0F0BD04F0C9FEECE7A9
:106C5000F7B5009308AB1B8807000C200D00160049
:106C6000019305F03DF8041E13D0280001F042FF07
:106C700000280FD00078D0232370C93BA370009B5D
:106C800021002381019B6770A580E680638105F068
:106C90007FF8F7BD014B1878EDE7C046F845FF1FB8
:106CA00013B5040064890389C2888188C078009480
:106CB000FFF7CEFF13BD000010B5044C206800287C
:106CC00003D005F005F80023236010BD9C67FF1F6B
:106CD000A122F0B5818892004A43384B384F1B6897
:106CE00004009B189D2292009B18827989B01A603B
:106CF0003B68002B5FD01D78324B1B68002B04D003
:106D00005B68002B01D00020984726000836310030
:106D1000E079FFF7B7FD237DE0710200E07804938E
:106D2000638A29000393238A0293E3890193A3884A
:106D300000933300FFF752FFE378002B0BD1E28979
:106D4000A379A18802920196E2792800009201229B
:106D500001F0DAFEE0703B68002B20D0FFF7ACFFBB
:106D6000194D287800281AD0184B1978FFF778FEAB
:106D7000002814D02B78E67808200793A78804F021
:106D8000AFFF011E09D0D0230370CA3B4670837049
:106D900087808671079804F0FBFF00232B70172172
:106DA000A088FFF775FCA08801F034FCA08801F0F2
:106DB0000BFD09B0F0BD064B9DE7C0463409FF1F2F
:106DC0009C67FF1FB067FF1F9167FF1F9067FF1F42
:106DD000F845FF1FF8B5070008000E0001F08AFE15
:106DE000041E18D02620FFF78DFC051E00D1257843
:106DF000062004F075FF041E0DD00021062204F0C9
:106E0000EFFDD0232370C23B21006770A370A680E2
:106E1000E8B204F0BDFFF8BDF0B585B001930AAB50
:106E20001B78070002930BAB1B7808000D00009243
:106E3000039301F05FFE061E22D0102004F050FFE5
:106E4000041E1DD01022002104F0CAFD2620FFF7E9
:106E500059FC002800D13078D0232370C13BA370A7
:106E6000009B21002372019B67706372029BA580C7
:106E7000A372039BC0B2E3720C9BE36004F088FF33
:106E800005B0F0BDF7B50D00019001F033FE071E0F
:106E900020D00E2004F024FF041E1BD02620FFF774
:106EA00031FC061E00D13E78D0232380C53B06224C
:106EB000A370F91DE01C04F033FF019B2A006381DD
:106EC0000123DD401A401D40210022736573F0B29A
:106ED00004F05EFFF7BD0000F0B585B00290100031
:106EE0000D0017000A9E039301F004FE041E31D02A
:106EF000029B002B2ED1039B02795B0724D5122322
:106F000013430422002E08D10B99002905D10C99B6
:106F1000002902D10D9900291AD01A430D9B227124
:106F2000002B00D0C9E0002E00D1CFE0002D00D012
:106F3000CCE0606A002801D004F0CAFE1C213000B9
:106F400004F076FF606205E002239A430E33D7E730
:106F500093432371654BBA00D458002C00D1AAE0AA
:106F6000002E10D0236A002B03D11C2004F058FE01
:106F700020625E4BBA00D358186A002803D01C2246
:106F8000310004F0CDFE0C9B002B12D0574CBB00FF
:106F90001D596B6A002B03D1162004F041FE686274
:106FA000BB00E358586A002803D016220C9904F05D
:106FB000B7FE0D9B002B11D04C4DBC006659B36A37
:106FC000002B03D1142004F02BFEB0622B59986AD9
:106FD000002803D014220D9904F0A2FE380001F01D
:106FE00089FD051E67D0414BBA00D358002B62D0F3
:106FF0001A6A3420002A00D11C389A6A002A01D06B
:10700000143080B20B9A002A01D01C3080B25B6A27
:10701000002B01D0163080B204F062FE041E4AD06C
:107020001822002104F0DCFC2620FFF76BFB019006
:10703000002801D12B780193D0232370029B2000DC
:1070400063700A23294EA370039BBD00A371AB5943
:10705000A780196A1830002905D01C22A06004F00E
:107060005FFE200034307359996A002907D003006D
:1070700014221433E060029304F052FE02980B9B3A
:10708000002B08D003001C221C330B9920610293B3
:1070900004F046FE02987359596A002903D016225B
:1070A000606104F03DFE6B462100187904F070FE2B
:1070B0003800FFF7E3FC05B0F0BD10220D9B0D99E1
:1070C0001B69A018236204F02BFE2CE70B9B002BFE
:1070D00000D13FE7012D00D03CE7606A002801D0D5
:1070E00004F0F6FD1C210B982AE7C0469867FF1FA5
:1070F00010B5044C2068002803D004F0E9FD0023FB
:10710000236010BD8C67FF1F0B4B07B51A68002A60
:1071100001D100200EBD6946531C012012780731B1
:10712000FFF772FC0028F4D0027801231000184009
:107130001A42EED0EEE7C046A867FF1FF0B51F4F1A
:1071400001203B6887B0002B25D09B78059300F089
:10715000B3FB002821D00A20FFF7D4FA04000B204B
:10716000FFF7D0FA164B05001E78731E9E413B6850
:10717000F6B2191DD878FFF757FB3B682900DA7A79
:10718000043303929A790193029200903300200015
:10719000059A04F0D5FB07B0F0BDFFF7B5FF002856
:1071A00005D00620FFF7AEFA04000720D8E7082034
:1071B000FFF7A8FA04000920D2E7C0468C67FF1F3A
:1071C0008867FF1F70B50A4E040033780D00FF2B4F
:1071D0000DD0042004F084FD011E08D0D0230370DC
:1071E000CE3B45708370C470307804F0D1FD70BD23
:1071F0000846FF1F70B5040006200D0004F070FD66
:10720000011E0AD0D0230370CD3B8370054B447020
:107210001B688580187804F0BBFD002C01D0FFF7B7
:1072200067FF70BD8C67FF1FF8B5264F06003B68EF
:107230000D001124002B05D10522234B1B7813428E
:1072400002D112242000F8BD204A10241268002A1E
:10725000F8D01278002AF5D0DB0719D52B789A1EC2
:10726000012A1AD80C2004F0DBFC13243860002813
:10727000E8D000230A22437029000670023004F08F
:107280004FFDFFF75BFF041E0AD0FFF731FFD9E780
:1072900000F012FB0028E1D1E4E7002BE2D0D0E7B8
:1072A0000B4B1B78032BCDD11D20FFF72BFA094B7D
:1072B00018800028C6D0084B04211878074A04F02B
:1072C0008FFDBFE78C67FF1F8967FF1FA867FF1F40
:1072D0008867FF1F8667FF1FB467FF1F60EA000013
:1072E000F7B50193194B14001A78052306000F0017
:1072F00012201A4221D0012920D1154B1D68002DE2
:107300001BD002201F2C18D8002C02D0019B002B70
:1073100013D0104B1F221E706E1C0021300004F091
:107320005FFB01992200300004F0FAFC31002000DC
:107330002C70002F06D004F0ABFAFEBD064B1220D5
:107340001D68DCE704F064FAF7E7C0468967FF1FB1
:10735000A867FF1F0846FF1FA467FF1FF8B50F4E61
:1073600012243368002B17D01B780F3C834213D1B3
:1073700000250B4F0221387804F042FC094B042110
:1073800038781D8004F03CFC074B28001D803368D2
:107390005C7004F06DFA04002000F8BD8C67FF1FDC
:1073A000B467FF1FA067FF1F8667FF1F70B5012826
:1073B00023D11B4C2388002B03D01A4A1578002DAB
:1073C00007D0194B1B68002B02D01878FFF7C6FFB7
:1073D00070BD3B2B02D93C3B2380F9E7134E0221C1
:1073E000307804F00DFCFA222388920002215A43DF
:1073F000307804F005FB2580EAE70B4B1B68002B77
:10740000E6D00B4B1B785B07E2D5084B02211878BE
:1074100004F0F6FB0022024B1A80FFF769FED7E763
:10742000A067FF1F8467FF1F8C67FF1FB467FF1FE4
:107430008967FF1FF8B51E4D2868002803D004F0A7
:1074400047FC00232B601B4E3068002803D004F05B
:107450003FFC00233360184F05243B781800204080
:10746000234221D0154800F02BFA3B78234213D059
:10747000202004F0D5FB2860002813D02022002112
:1074800004F0AEFA202004F0CBFB041E306005D0DF
:107490002022002104F0A4FA002004E0286804F06F
:1074A00017FC2C601320F8BD00F00AFAF4E7C04680
:1074B000A867FF1FA467FF1F8967FF1FFC45FF1F09
:1074C00010B50A4C23681A1E0ED0002808D10130CE
:1074D000587004F0CDF9002805D02368002B02D0A5
:1074E0000021FFF787FE0122100010BD8C67FF1FEF
:1074F000F7B5274E050033680191181E21D05C783E
:10750000244F012C30D1FFF7FFFD002825D02000AB
:10751000FFF7F8F80400412814D91F4B022118780E
:107520001E4A04F05DFC1E4B3C3C1C80022233686A
:107530005A703B78002B14D128000199FFF75AFEAE
:107540000120FEBDFA2292004243002AEED0124BE7
:107550000221187804F054FAE8E7FFF7D3F80200A4
:10756000F3E700233B70EBE73B78002BE8D10320E7
:1075700004F0B6FB011E08D0D0230370CC3B45704D
:1075800083703368187804F003FCFFF7B1FDD7E788
:107590008C67FF1F8467FF1FB467FF1F60EA00004E
:1075A000A067FF1F10B51749838802008B4220D0C7
:1075B00011D815498B4217D0144900205B1899B295
:1075C000012907D8926811785A425341D8B2FFF77F
:1075D000F9FD012010BD0E4A00209B1807229BB226
:1075E0009A424041C0B2F5E783681878FFF768FF18
:1075F000F0E7836899785A78090218781143FFF701
:1076000077FFE7E70A20000006200000F8DFFFFF11
:10761000AFDFFFFF014B18707047C0460946FF1FE0
:1076200010B5064C207001F041FA207804F050F9B2
:107630000521207800F062FD10BDC046B467FF1F31
:107640000BB273B50D00002B00DBC4E0884B18783B
:1076500004F056FB041E0ED00378912B0FD0A22B02
:1076600000D1A1E0834B1878FF2852D0210004F00C
:107670008FFB00284DD180200002684076BD437802
:107680000F2B76D013D8052B70D00E2BEAD1808823
:10769000794B98422BD8794B98421BD8784B98421B
:1076A000E0D1A3681878591CFFF774F838E03E2B36
:1076B000D8D18378032B74D06CD8012B6ED0022BD9
:1076C000D0D1704B1B68002B23D05B68002B20D0DF
:1076D00098471EE06C4BC0180C28C3D804F030FB50
:1076E0001DC2C2150BC20B0B0B3223C23C00674BF1
:1076F000C0180728B6D8664B1B68002B09D01B683A
:10770000002B06D0200098470AE0A3681878FFF7FE
:10771000C7F8200004F0ACFAADE7A068FFF762F804
:1077200000289FD0F5E7A3681B78002BF1D0554BBC
:107730001B68002BEDD01B68002BEAD021005548B8
:107740009847EDE74F4B1B68002BE2D01B68002BDE
:10775000DFD021005048F3E7504B1B68002BD8D0F6
:107760005B68002BD5D021004348E9E7FFF7EAF931
:10777000CFE780884A4B984203D04A4B984200D0CA
:1077800070E7464B1B68002BC3D05B68002BC0D052
:107790002100D5E7153B012BBBD963E7FFF798FA2A
:1077A000B7E7FFF77DFAB4E73F4B1B78042B07D10F
:1077B00000236A4613800179408800F0C5FCA8E7E1
:1077C000364B1B68002BA4D05B68002BA1D00100B6
:1077D000364898479DE7012421420AD0294B1B686F
:1077E000002B04D05B68002B01D0002098470120BB
:1077F00043E78B070AD5264B1B68002B04D05B6838
:10780000002B01D020009847022036E704212800F1
:1078100008400D4200D131E7254E3388002B21D09E
:10782000013B9BB23380002B1AD1FFF7DBF8002815
:107830000AD0204B1C70164B1B68002B04D05B68D1
:10784000002B01D020009847FFF7C6F8694601F0E9
:1078500001FD6846FEF7FEFF1D20FEF753FF308056
:1078600004200AE7024B187804F0CAF9F8E7C0468A
:10787000B467FF1F0946FF1F0E2000000120000013
:1078800009100000AC67FF1FFEDFFFFFAFDFFFFF47
:10789000B067FF1F0C2000000B2000009467FF1F43
:1078A0000D200000132000008967FF1FFFFF00006C
:1078B0008667FF1F8467FF1F10B501F09BF910BD9D
:1078C000014B18607047C046B067FF1F0B8800204F
:1078D000162B01D817230420014A13807047C04695
:1078E0005E67FF1F00207047074A0300118881422E
:1078F00007D091880020994202D1013080001018F1
:1079000070470020FAE7C046BC67FF1FF0B58F78CC
:1079100006000D00C7B01E2F15D1FFF7E5FF051EAD
:1079200003D10024200047B0F0BD00223B0031000D
:10793000C078009200F0B2FB0400A81C00F0D3FB5A
:10794000FF23EB70EEE7264B062403931B78FF2BF7
:10795000E8D0182FE6D87B08224A013BDB000292D0
:107960009A589446002ADDD0029AD3185B68002BFF
:10797000D8D00878002802D14B78012B02D10624F8
:10798000122FCFD107AFAB88697800976446AA68F9
:10799000A047041EC6D1AB78029A5B08013BDB000E
:1079A000D318390030005B689847041E0BD1AB78C0
:1079B000042BB6D0039A310010782200009700F013
:1079C0006DFB0400AEE76A78002AABD1AA7805A95E
:1079D0003B88087130000A704B80FEF747FBA0E738
:1079E0000C46FF1F58C000111D4B37B505009842CB
:1079F0000BD000290AD1FFF777FF002805D11948DD
:107A0000FFF772FF002800D0058037BD01291AD189
:107A1000FFF76AFF041EF8D001235B420380A378BE
:107A2000FF2BF2D0FE2B07D00023E0781422009326
:107A300029001E3300F032FBA01C00F054FB012390
:107A40005B426380E1E70229DFD1013901F0BEF832
:107A50000028DAD12800FFF747FF041EDFD1D4E762
:107A6000FEFF0000FFFF0000022210B5074B52424C
:107A70001A80074801325A809A80DA8000F07EFA34
:107A8000044801F025F8002010BDC046BC67FF1F68
:107A90000D790011E97900110388F7B50400002B76
:107AA00002D102252800FEBD426802211378254834
:107AB0005268FEF7A5FD00282ED0234F01253A88F5
:107AC000002AEFD0802321885B0201259B1A99426E
:107AD000E8DC0C2004F0A4F8061E31D03B88228894
:107AE0009C4600231800019561469DB2491989B250
:107AF000AA421BD8002801D062443A8000233000FB
:107B0000082208C0210004F00BF9104A1368002B6A
:107B100013D100251660C5E76268022113780C486E
:107B20005268FEF76DFD0028C7D1BAE760681D01F5
:107B30004019418101330198D6E71A001B68E6E736
:107B40001325AFE7C6C000110A46FF1FB867FF1F25
:107B5000C4C00011014B18707047C0460C46FF1F8F
:107B600014230A0010B51A40194204D00122102132
:107B700001F048F810BD4B06F9D4012088434000BD
:107B8000F8E710B514008B0604D50122102101F08E
:107B900039F810BD08230A001A40194202D14BB22D
:107BA000002B0FDA102101F02DF8002808D0230057
:107BB000F9331B78002BECD0F8342378012BE8D173
:107BC0000020E6E703208907FAD4E2E7F0B51F00BA
:107BD000184B85B01C68019002910392002C27D1AC
:107BE000200005B0F0BDA5683301ED186B89019A3E
:107BF000934211D3029A93420ED8002F04D10A9BCC
:107C0000002B10D12C00EBE73B002978039A686821
:107C1000FEF7F6FC0028F2D10136B6B2A388B342D3
:107C2000E1D82468DAE7A3680A9A5B891380E9E758
:107C30000026F3E7B867FF1F37B50C000A884988AC
:107C40000123914217D3002A15D0651D23792A00FC
:107C500002210A48FEF7D4FC102300280BD0237918
:107C60006188208800242A000094FFF7AFFF0A23D0
:107C7000A04200D0230018003EBDC046C6C000117F
:107C800013B50A0008884988012388420BD80028C8
:107C900009D00024137905320094FFF797FF0A23D7
:107CA000A04200D02300180016BD13B50A000888B2
:107CB0004988012388420BD8002809D00024137971
:107CC00005320094FFF782FF0A23A04200D0230070
:107CD000180016BDF0B58BB003904A8808880E00D6
:107CE0000123824255D3002853D00023012704AC3E
:107CF00023700022718813000092FFF767FF051EB2
:107D00003ED02078002835D12B78022B18D167700F
:107D10006A8983000130E31880005A806968022272
:107D2000201803F0FDFF23780133DBB22370042B0E
:107D300019D93B006889013080B2002BD9D01FE0EF
:107D400002236370122358436A89231804305A802F
:107D500069681022201803F0E3FF23780133DBB2B7
:107D60002370002BE5D10C4A6B899B185A42534172
:107D7000DBB2DFE76378012BE4D12B78022BC7D08D
:107D800022780A23002A04D021000398FEF798F9EC
:107D9000002318000BB0F0BD0100FFFF0F4BF0B542
:107DA00004001868002816D083685D89A54207D8AA
:107DB0008288AE18B44203DA12019A18934201D1B4
:107DC0000068EFE71E005F891036A74204D1002942
:107DD00000D00D801800F0BD3300EFE7B867FF1F3B
:107DE00070B505000C0008880021FFF7D7FF0300DD
:107DF0000120002B04D022002800197AFFF7C1FED1
:107E000070BDF7B50C00002501902300F6331B78F8
:107E1000AB4201D800200AE06B00E65A0021300096
:107E2000E718FFF7BBFF002802D126800130FEBD16
:107E3000017A0198FFF794FE002802D03B88238046
:107E4000F5E70135EDB2E0E710B504000888002140
:107E5000FFF7A4FF03000120002B03D02000197AB4
:107E6000FFF77EFE10BD0000054B1B68002B01D103
:107E7000180004E09A6852898242F6D198887047C7
:107E8000B867FF1FF0B50E27002687B0039302AB3B
:107E9000FF183E8005001F4B40891400984207D010
:107EA0002B78013000976A6880B2FFF78FFE0600DA
:107EB00002212B7818486A68FEF7A2FB00280FD031
:107EC0006C892000FFF7D0FF002802D0013C041984
:107ED000A4B2039B002B00D01C80300007B0F0BD83
:107EE00002212B780D486A68FEF78AFB0028E7D14B
:107EF00002212B780A486A68FEF782FB002807D027
:107F0000002EDED03B88A342DBD17489013CDFE741
:107F10006C89DEE7FFFF0000C6C00011C4C000117D
:107F2000C2C0001110B50C00FFF7DEFC03000220F8
:107F3000002B0AD0002C00D023609B781720FE2B4A
:107F400003D00138FF2B00D1002010BD73B50D0008
:107F500001A904001600FFF7E5FF172805D0002E41
:107F600004D129002000FEF727F976BD0122102157
:107F7000200000F047FE0028F3D0F6E7014B186020
:107F80007047C046C867FF1F37B56B469D1D01008F
:107F900004000222280003F0F3FD2B88B02B0ED141
:107FA0002379122B09D12300FF339B78012B06D1B3
:107FB0000121608800F0E0F801E01B2BF8D037BD0C
:107FC00010B5054B0421187000F098F8FFF74CFD30
:107FD000FEF770FB10BDC046CC67FF1F0020F0B558
:107FE0000BB20F0087B0834234DA274B187803F0C6
:107FF00087FE051E2BD00378A02B25D103AE3100C0
:10800000FEF7E4F8041E0BD1B378DB0724D51F4B31
:1080100006341B68002B03D03100688898470400A1
:10802000A868002801D003F03BFE002C08D1184AB4
:10803000039B1340174A934206D0B3781B2B03D0FF
:108040000121688800F098F8280003F011FE8020D4
:108050000002784007B0F0BD0F4B1B68002B10D01A
:10806000310068889847041EDAD07378002BD7D186
:10807000B27801A90A704B800C716888FDF7F6FF91
:10808000CEE70624F1E7C046CC67FF1FC467FF1F99
:1080900000FFFF0000011200C867FF1FF7B5019045
:1080A000822040000D0017001E0003F019FE04009E
:1080B0001320002C12D0B02320002370089BFC2238
:1080C0006770658026710830002B08D0190003F016
:1080D00027FE2100019803F05BFE0020FEBD0899F9
:1080E00003F07EFCF5E710B5041E06D00078FD28ED
:1080F00003D803F06DFDFF23237010BD0A1F93B258
:1081000010B504000220032B05D882400020024B4A
:10811000D1529B189C7010BDEC67FF1F0B8870B587
:10812000043B04000D000220032B0BD8012120008A
:1081300000F04CFD03001420002B03D02900200088
:1081400000F0DEFB70BD000007B51300034A00928B
:108150000A00012100F02CFC0EBDC04685830011F1
:1081600007B5019203220092024B0A00122100F08F
:1081700049FC0EBD0384001107B56B4601AA1180AE
:108180000449D88008780633012802D1190003F089
:1081900007FE07BDCD67FF1F0C4B10B518700023FD
:1081A000FF210B4A1380138193819380094A5380E6
:1081B0001370517293819372D174D3821375517776
:1081C00003F066FD00F0FCF910BDC046FC67FF1F20
:1081D000EC67FF1FCE67FF1FF0B58DB06B46002028
:1081E00003910C229B5E834200DBB0E05D4B18786C
:1081F00003F086FD051E00D1A4E00378902B00D08B
:108200009DE006AF01004688380000F013FA796857
:108210000400002900D19CE03B88052B6ED13B89EE
:10822000032B1CD905AC200000F0A2F86288172AA5
:1082300061D83989131D994231D179682378043185
:108240000291D90738D5607800F08EF9071E06D064
:10825000002303712378012B08D0132B23D0A868A7
:10826000002800D178E003F01BFD75E062880299D8
:1082700009A800F0A6F80290380000F08BF909AACE
:108280002378387A0192002231000092029A00F09D
:1082900012F9380000F064F9029B002BDFD03000A7
:1082A00000F080F9DBE70378032BD8D162880299CC
:1082B00009A800F0D6F8DEE7122B13D1029909A81D
:1082C00000F0B5F8021EEAD127498B88002BC6D0F2
:1082D000887909A92378019161780091310000F033
:1082E000EAF8BCE7002302AA93833000617809AA68
:1082F000FFF72AFFB3E71D4B0993F6E7042B02D0E3
:108300009A1F012AABD8184A043B9B00995A0029AE
:10831000A5D0D218907831003A0000F0AEF80028CD
:108320009DD13B88042B03D001213000FFF724FFAF
:10833000012C04D1A868002801D003F0B1FC28006A
:1083400003F096FC8020039B0002434018000DB010
:10835000F0BD012800D182E701213000FFF70CFFBA
:10836000EDE7C046FC67FF1FEC67FF1F0100170029
:108370000B7803704B784370CB788A781B021343D9
:10838000438070470A88030002700A88120A42700C
:108390000A88012A06D14A8882704A88120AC27065
:1083A0000420704702208242FBD14A8804309A7030
:1083B0004A88120ADA708A881A718A88120A5A71EF
:1083C000EFE710B50400012082420CD94B780A78FF
:1083D0001B0213432380834206D1CB788A781B0289
:1083E00013436380002010BD022BFBD1CB788A7829
:1083F0001B02134363804B790A791B021343A3804A
:10840000F0E70B8803700B881B0A43704B8883705E
:108410004B881B0AC3708B8803718B881B0A4371BE
:10842000CB888371CB881B0AC37108207047030077
:108430000120082A14D14A780878120202431A80CF
:10844000CA788878120202435A804A79087912025F
:1084500002439A80CA798879120202430020DA80A6
:10846000704710B504000120022A05D100204B7886
:108470000A781B021343238010BDF8B506001020B4
:108480000F00150003F02CFC04000120002C0ED07E
:10849000A0230C22290023806780201D002D07D0F7
:1084A00003F03EFC2100300003F072FC0020F8BD18
:1084B00003F096FAF6E7F7B51E00009008AB14201B
:1084C00017001D78019103F00BFC041E12D0A223AB
:1084D0000370019B47704380099B057146710C2214
:1084E0000830002B07D0190003F01AFC2100009877
:1084F00003F04EFCF7BD099903F072FAF6E737B5C1
:10850000041E0FD04388002B0CD00025C1881323F4
:10851000007A172201950095FFF7CDFFFF236580B4
:108520006372257037BD000010B50C4904004A88FD
:10853000002A09D08B89002B05D00020CB8A02228B
:10854000834201D010BD012213000A2043430020C2
:108550004032C854C81842800472F3E7CE67FF1F48
:108560000023438003707047094B00211A0010B5A7
:108570005C88002C06D01C79844203D10A234B432B
:10858000D01810BD01310A330329F1D10020F8E7DA
:10859000CE67FF1F10B50400407A03F019FBFF23DC
:1085A000637210BD7047043010B580B203F088F9D3
:1085B000002803D00421494203F04AFB10BD00000B
:1085C00070B50025104CA0682580A581A580A84223
:1085D00002D003F065FBA56000250C4C0C4B606DD0
:1085E0001D80230058331D70A84202D003F058FBB1
:1085F000656500256068002801D003F051FB013556
:1086000008340A2DF6D170BD9468FF1F3868FF1F2B
:108610008868FF1F70B5041E09D1054D2880A88108
:10862000A880A868002802D003F03AFBAC6070BDB7
:108630009468FF1FF0B54B8885B001930023436019
:108640000A7905000F00022A00D07BE0CA88032ABD
:1086500017D98B685E7819783602DC78D8790E43A2
:1086600099781B7A24021B020C43034353495BBADB
:108670000B80331D93421ED1042C04D0631F022BA8
:108680000ED9012015E0019A4D4B1201D35A002B4F
:1086900006D00198FFF7BEFF4A4A13690133136100
:1086A0000421B8682E812C80494203F0D1FA686019
:1086B000002005B0F0BD434D042C06D0631F022BF3
:1086C0000FD9EB680133EB60DBE7019A3C4B1201F9
:1086D000D35A002B05D00198FFF79CFF2B6901337B
:1086E0002B61374B30000293019B029A1B010193CF
:1086F000002301998C468B52130063449C800393A2
:108700009E81FFF750FF039B041E986016D0042142
:10871000B868494203F09CFAFA880100043A200044
:1087200003F0FEFA0199029AFB888A5A043B9B18CF
:10873000029A8B522B6801332B60A2E7AB6901339D
:10874000AB619EE71E4B0293019B1E01029BF35AF5
:10875000002B2DD002998C19A068002828D0012A5E
:1087600026D1FA889B189BB27352A189994217D3DC
:108770009B1AC018B96803F0D3FA029BA289F35A76
:10878000934200D07DE700222B81A3882B80A36831
:108790006B60029BF2520B4A53680133536070E7DF
:1087A000084A9368013393600198FFF733FF68E745
:1087B000044A536901335361F6E7C046FE67FF1F61
:1087C0009468FF1F0468FF1F70B5051E15D10B4C80
:1087D0000B4B1880230058331870606D002802D0AE
:1087E00003F05EFA6565250050356068002801D009
:1087F00003F056FA0834AC42F7D170BD3868FF1F59
:108800008868FF1FF0B51700A12285B09200019380
:108810004243394B06001B680C009B18D933FF33C9
:108820001D78FDF741FF0430854204DD3000FDF77F
:108830003BFF0430C5B2BD4207D33A0000213000EF
:10884000019B03F085F805B0F0BD2900380003F066
:10885000BFF82300C6B250331E700393019B29005A
:108860006365380003F0FCF9CBB20293002B02D011
:10887000039B01361E7000262300503303931B78A0
:10888000B34204D8606D002831D10020DBE7029AA2
:108890002800002A04D0013B1000B34200D0280079
:1088A000F700E719387003F03BF8786000280ED025
:1088B0003A78019903F034FA019A3B780136D318DB
:1088C0000E4A0193D369F6B20133D361D4E7039B17
:1088D00018706065A74205D1084A1320D36A013396
:1088E000D362B0E7606803F0DBF90834F2E703F025
:1088F000D7F900236365C8E73409FF1F0468FF1F29
:10890000F7B50D0007000421686803F0A1F92B8971
:10891000040003702B891B0A43702B8883702B88FB
:108920001B0AC3702E8902250436F6B2FB2E15D819
:108930001B4B9F4214D10C2003F0D2F91135011EBC
:108940000CD0902303708E3B0371043B4380154B86
:108950008460C680187803F01BFA00252800FEBD4D
:108960005C237B43104AD3180093583301931B7840
:10897000002B0FD10300320038000099FFF742FFAF
:10898000019B05001B78002BE8D13800009903F00B
:10899000E7F9E3E7054A0725536A01335362DDE748
:1089A000FEFF0000FC67FF1F3868FF1F0468FF1F01
:1089B000F0B587B0009017200F0016000193FFF765
:1089C000F2FD1325041E19D00C98031E02D0019944
:1089D000201D9847030AE370052302AAA070043003
:1089E000908127700098667003A993800494FFF724
:1089F00087FF051E02D0200003F052F9280007B0BF
:108A0000F0BD0000F0B587B01F000CAB1B780391E0
:108A1000059301210DAB06001C78049200F0D6F8F6
:108A20001425002821D02000FFF77EFD0135041E0B
:108A30001BD01149059B0A7803700132D2B2131E74
:108A4000C68001D101231A000B7022713000049BF3
:108A500003990097FFF7ACFF051E09D12300210001
:108A60000648074A093302F09BFF280007B0F0BD13
:108A7000002363802370F8E70068FF1FFF84001164
:108A800030750000F8B505000E00064C064F23684F
:108A9000002B02D03100280098470434BC42F6D1A4
:108AA000F8BDC046A468FF1FB868FF1F0123064A2F
:108AB0005B425380002313715362044A1360536076
:108AC0009360D36013617047B868FF1FA468FF1FED
:108AD0000200002310B506499C000859002801D166
:108AE000625010BD0133052BF6D11320F9E7C046C3
:108AF000A468FF1F034A5388181A43425841404252
:108B000010407047B868FF1FF0B585B002930AABFC
:108B10001F780CAB1B88009008000E000192039395
:108B2000FFF7E8FF05001120002D1BD10E48FFF7CD
:108B3000E1FF04001520002C14D006220B99A77128
:108B4000E01D03F0EDF8019B30002371029B29002A
:108B50006371009B66802370039B6562E381FFF76E
:108B600091FF280005B0F0BDFFFF000010B5FFF732
:108B7000C1FF04000220002C12D060880121FFF701
:108B800081FF606A002801D003F0A2F828220021AA
:108B9000200002F025FF012300205B42638020714A
:108BA00010BD000030B5074A074C55880100137806
:108BB0000020A54204D05B1A59424B415842104054
:108BC00030BDC046B868FF1FFFFF0000084A10B55F
:108BD00001230C00904208D0FFF78CFF031E04D045
:108BE000037923405A1E9341DBB2180010BDC046E2
:108BF000FEFF0000024B1879431E9841C0B2704737
:108C0000B868FF1F70B504000D001600FFF772FF73
:108C1000002804D10D4B9C4200D0143070BD416A35
:108C200003790520002907D012221A40102A02D108
:108C30000520002EF2D10F20DB06EFD5897E0C2017
:108C4000A9428941494249420840E7E7FEFF000046
:108C5000030010B5002800D110BD0348034A418825
:108C60009142F9D09847F7E7B868FF1FFFFF00006F
:108C7000002330B5C45CCD5C6C40D4540133102B60
:108C8000F8D130BD0F23002210B5C45C640022432C
:108C9000CA54C25CD209013BF7D210BD02000100E8
:108CA00010B52032103103F053F810BDF0B58BB081
:108CB0000390102005931700049102F0B1FF00907B
:108CC000102002F0ADFF009B13240190002B05D073
:108CD00000280CD11324009802F0FAFF019B002B0E
:108CE00002D0180002F0F4FF20000BB0F0BD1020FD
:108CF00002F096FF0600102002F092FF13240500F8
:108D0000002E00D1AEE0002819D01022002102F080
:108D100067FE32002900039803F01AF8041E0ED1F2
:108D200033787F2B51D830000099FFF7ABFF009BC1
:108D30001B787F2B53D801990098FFF7A3FF3000D1
:108D400002F0C6FF002D02D0280002F0C1FF002C67
:108D5000C1D1102002F064FF0600102002F060FF75
:108D60000290002E7CD0002878D03A000F322300E9
:108D70000125121105D00F333B4015B25A42534121
:108D80001BB26A1E1201002B33D0049BD2B298187A
:108D90000099029AFFF76CFF013D1022002130007C
:108DA00002F01EFEADB2049F2D017D19AF4242D0EC
:108DB000002C33D0300002F08BFF029B002B00D13F
:108DC00089E7180002F084FF85E729003000FFF7EB
:108DD00059FF28002549009AFFF74AFFA7E7290015
:108DE0000098FFF74FFF28002049019AFFF740FF46
:108DF000A5E70F210F4004998A18D9B28F4208D9EC
:108E0000D15C06A819540133102BF6D1029A0199AE
:108E1000C0E7791A48424141C901F2E73900300000
:108E200006AAFFF725FF3200039806A902F090FF7B
:108E300010370400BAE7002CBCD13000029906AA12
:108E4000FFF716FF320006A9039802F081FF0822FF
:108E500004003100059802F063FFABE71324A9E793
:108E60001324AAE7002800D06EE733E7CCC0001136
:108E7000F0B58BB00F0016000225009000283FD0FF
:108E8000002A3DD00B1DDBB21800029302F0C8FE91
:108E90001135041E34D0FDF747FD05003A00009956
:108EA000201D02F04DFEEBB20393E3702B0CDBB2FE
:108EB0002F0A00936370FFB22B0E2370A7700193EB
:108EC000FDF72CFD1022010006A802F039FE21005A
:108ED000029A04AB06A8FFF7E9FE051E0DD1039B1D
:108EE00008223370009B04A9B370019B7770F37064
:108EF000301D02F025FEFDF71DFD200002F0E8FE0A
:108F000028000BB0F0BDF0B58FB00D00149E03909B
:108F100004920593002A03D1022420000FB0F0BD73
:108F2000002EF9D00398FFF7E5FD1424071EF4D0B6
:108F30007278337812021A43B3781B041343F27821
:108F400012061A43036A0192934201D30133E3D11B
:108F5000002D03D03B7901249B07DED50822002198
:108F600006A802F03DFD059B13240433DBB2180074
:108F7000029302F055FE051ECFD0059A04990430E5
:108F800002F0DEFD04223100280002F0D9FD390094
:108F9000102210310AA802F0D3FD2900029A06AB74
:108FA0000AA8FFF783FE041E0FD1082206A908A80D
:108FB00002F0C6FD0822311D08A802F089FD012833
:108FC00007D101990398FDF7C9FC280002F080FE43
:108FD000A3E70124F9E7000070B51C4C05002368E5
:108FE000181E10D0002D14D11A78002A0CD1981C0C
:108FF000083202F095FE02F0FBFE0135002808D190
:1090000023681D70012070BD0A331800082202F089
:1090100087FE2368002BF5D0122002F061FE061EA9
:109020000DD0C12321680370457002311022023037
:1090300002F076FE23683100587802F0A9FE20681D
:1090400002F046FE00232360DCE7C046E068FF1F15
:10905000F8B504002020FDF755FB0D4EA700BB59C5
:109060000500002B0DD000280BD0D878FF2809D19F
:1090700008492A000C55F35907480333611802F0D8
:109080008FFCF8BD290002F073FE0028F0D1F8E74C
:10909000FC68FF1FE468FF1FA9A2001170B5064D10
:1090A00084006359002B05D0D87802F091FDFF228F
:1090B0006359DA7070BDC046FC68FF1F70B50600CA
:1090C0008CB00C00150000213022684602F088FCAC
:1090D00031001022684602F033FD1D2021000322DA
:1090E000684402F02DFD6846FFF7D8FD2D210400ED
:1090F00003222800694402F023FD20000CB070BD5B
:10910000F0B50700160097B001931CAB1D78302214
:109110001EAB00910AA800211C7802F061FC10220D
:1091200039000AA802F00CFD1022002102A802F06A
:1091300057FC0722310002A802F002FD072202AB11
:109140009818631E9C41019902F0FAFC02AB9C73D3
:109150002B005A1E934102AAD3730021102206A8A5
:1091600002F03EFC06221D9907A802F0E9FC1A2035
:1091700002ABC01806221F9902F0E2FC10220099EF
:109180000EA802F0DDFC102202AB0EA908781C78B4
:10919000013A6040D2B2087001330131002AF5D1A2
:1091A0000AA8FFF77BFD102212A904000EA802F006
:1091B000B7FD102206AB0EA908781D78013A684069
:1091C000D2B2087001330131002AF5D10AA8FFF7A5
:1091D00065FD044310222098E4B212A902F0B0FC0D
:1091E000200017B0F0BD70B50E0014008CB0010067
:1091F000102268461D0002F0A3FC3100082204A8DA
:1092000002F09EFC2100082206A802F099FC6846A4
:10921000FFF744FD04001022280008A902F090FC8A
:1092200020000CB070BDF8B506000D000024371901
:10923000AC4200D3F8BD02F0CBFD030A3B70631CC7
:10924000DBB201379D4203D90234F054E4B2EEE7B9
:109250001C00EDE773B506000C000225002819D0AC
:10926000002917D0032101A8FFF7DDFF6B469A798B
:109270003F231A40013313436A463000937101A91A
:109280002200FFF71BFF051E04D10322E01C01A9E9
:1092900002F046FD280076BD03785807DA08C00FB3
:1092A000D20080009B0710439B0F1843C0B2704749
:1092B00007230B40C908C9000B4303707047000027
:1092C00070B50400FFF7EAFE134DA4006359002BAC
:1092D00021D0186A002801D002F0FAFC2B59986EB0
:1092E000002801D002F0F4FC2B59D86E002801D0E0
:1092F00002F0EEFC2B59186F002801D002F0E8FCB8
:109300002B59586F002801D002F0E2FC285902F0D6
:10931000DFFC00232B5170BDFC68FF1F0E4B80004B
:10932000C35870B50C00002B0FD09D68002D0CD0D9
:109330002B78201D0B706B784B70A97CFFF7B8FF62
:109340002B7E23726B69E36070BD10220021200028
:1093500002F046FBF8E7C046FC68FF1F014B1860AF
:109360007047C046F868FF1F074A03008000825814
:1093700010B5002A06D0D088984203D1012901D126
:10938000FFF79EFF10BDC046FC68FF1FF0B5264EDC
:1093900095B087000B93BB590500099112200A92E2
:1093A000002B31D0D888FFF7A5FB04001420002C37
:1093B0002AD0280010A9FFF7B1FFBB591E781D6AFB
:1093C000002E23D00895FDF7EFFA07000020FDF7E7
:1093D000F1FA0790A379E61D069310AD0CA9089841
:1093E00000F0E2FA0EA9280000F0D7FA0B9B0A99C8
:1093F0000493069B09980293079B03960193009799
:109400000EAB0CAAFFF77CFE15B0F0BDFDF7CCFA51
:1094100006903000FDF7CEFAE31DA779079310AB55
:1094200006000893DAE7C046FC68FF1F30B50C4C15
:1094300085002A59030085B00120002A0ED01800AB
:109440006946FFF76BFF2B591A78D888054B002A1D
:1094500000D1054B6A46072100F0D9FB05B030BDAD
:10946000FC68FF1F9B990011A999001130B5094CA8
:109470008500295985B010226846253102F050FC3C
:109480002A591121044BD0886A4600F0C0FB05B070
:1094900030BDC046FC68FF1F459A001130B5094C2D
:1094A0008500295985B010226846353102F038FC14
:1094B0002A591121044BD0886A4600F0A8FB05B058
:1094C00030BDC046FC68FF1F839A0011F7B54D4FB1
:1094D00086001020F4590D0002F0A2FBF35920621F
:1094E000186A132200286CD0033A29009C6802F005
:1094F00017FCF3591A780192002A58D11E6A227D6E
:10950000317B944651400122019F114201D16746AF
:109510001740217D914339432175377B4F40BC462D
:1095200060460027800701D44F0817400121022020
:109530008F40227D82433A432275377B5740BC4699
:1095400060460027400701D497080F400420227D81
:10955000BF0082433A432275627D002794466046ED
:10956000727B42400A4201D167460F400121627D71
:109570008A433A436275777B5740BC466046002772
:10958000800701D457080F400220627D7F0082438C
:1095900017436775767B00227E40760701D4BA08B0
:1095A0000A400426617D9200B1430A4362756A78DD
:1095B000002A08D06278002A05D005220533DA7720
:1095C00000221000FEBD04222979114205D1A17CA0
:1095D000114202D10533033AF1E7019A21782C7840
:1095E000002A02D10A002100140018220429E8D818
:1095F000042CE6D805206043034A05331218525C58
:10960000DDE7C046FC68FF1FDCC0001110B50A0092
:109610001121024B00F0FBFA10BDC046DF9A001189
:109620000B0030B587B001AD2B806B4604001100F4
:10963000981D082202F074FB2A000B212000024B27
:1096400000F0E5FA07B030BD079B001110B50A0025
:109650001121024B00F0DBFA10BDC0465B9B0011EC
:1096600013B50B0011006A4613706B460400062206
:10967000581C02F055FB6A4608212000014B00F0FF
:10968000C6FA13BD7B9B001110B50A001121024BD5
:1096900000F0BDFA10BDC046CB9B00117FB50500A0
:1096A0000B4BAA00D4580800002C0FD0666F237F04
:1096B000E28821780396266F0296E66E0196A46EE4
:1096C0000094FDF709FC2800FFF7FAFD7FBDC046B6
:1096D000FC68FF1F10B51721FFF7E0FF10BD000069
:1096E00070B50A000D00064B0221040000F08FFA4D
:1096F000060029782000FFF7D1FF300070BDC0467A
:10970000AB9A001170B586B000236A461370836867
:1097100004001D78681E0A2859D801A902F088F8AB
:10972000060633373B3F43474B4F5300180000F0CA
:1097300042F9062312284BD000281BD16088FFF77E
:10974000D9F90823002813D04279002A47D1264BA3
:109750001A78072312070BD5244B1A680723002A0F
:1097600006D01668002E03D0290001AAB0470300D6
:109770006A4613706B461B786088002B2AD1FFF76E
:1097800067FC06B070BD180000F06CF9D4E7180053
:1097900000F087F9D0E7180000F093F9CCE7180043
:1097A00000F0ADF9C8E7180000F0C3F9C4E71800ED
:1097B00000F0F6F9C0E7180000F0F6F9BCE7180071
:1097C00000F013FAB8E7180000F013FAB4E7072323
:1097D0006A46137069466088FFF782FFD1E7052368
:1097E000012AC5D1024BB8E78967FF1FF468FF1F44
:1097F000F868FF1FF8B52C4F8600F35904000D00E0
:10980000002B40D0DA8882423DD15A78062A33D1E3
:109810001A78002A2ED0012099681A6A097D01421F
:1098200006D0157B054203D007225A700120F8BDEF
:109830000220014204D0157B054201D00922F4E741
:109840000420014204D0127B024201D00B22ECE73B
:10985000164B1B68002BE9D05B68002BE6D020007C
:109860009847BB5900215B78122BDFD12000FFF70E
:1098700015FFDBE70E4BECE7112A04D1002900D0DD
:1098800032252900F2E7002D08D12000FFF732F938
:10989000002803D01023027913430371210028000C
:1098A000FDF798FAC2E7C046FC68FF1FF468FF1F87
:1098B000F868FF1F70B50E4E8500AB590400002BF1
:1098C00013D01B78002B11D10A4B1B68002B04D03E
:1098D0005B68002B01D02000984773595B78122BEE
:1098E00003D100212000FFF7D9FE70BD024BECE749
:1098F000FC68FF1FF868FF1FF468FF1F094B80001A
:10990000C3581020002B0CD01A6A002A09D09B687B
:10991000002B06D0127A1B7E101C9A4200D9181C0C
:10992000C0B27047FC68FF1F70B503000D00140043
:109930000220002A30D000292ED013700B78081D89
:1099400053704B789370FFF7A7FCE0700120022161
:109950002B7A23716B7B034063716A7B0A4013434C
:10996000042263716E7B1640334363716E7BF6088D
:10997000F600334363712B7B0340A371287B0140C6
:1099800000200B43A371297B0A401343A3712A7B58
:10999000D208D2001343A37170BD10B50A000100B4
:1099A0000120FFF7C1FF10BD10B50A000100022021
:1099B000FFF7BAFF10BD70B506000C000220002EA4
:1099C00030D000292ED07378201D0B70B3784B70E7
:1099D000F178FFF76DFC01223579257271794B1012
:1099E000080013409340104003438810104080004B
:1099F000C9080343C9000B436373B1794B100800D6
:109A00001340934010400343881002409200C9085D
:109A10001343C9000B4321202373FCF773FE8542D7
:109A200001D2122070BD2220257AFCF76BFE854200
:109A3000F7D823781820042BF4D86378012BF1D8B9
:109A40000020EFE7030010B50220002909D0002B09
:109A500007D00322481C0A7019000D3202F060F989
:109A6000002010BD03000222080010B5002B06D014
:109A7000002904D00E32591C02F052F900221000C5
:109A800010BD030010B50220002909D0002B07D01B
:109A90000422481C0A7019000C3202F041F900201F
:109AA00010BD10B5FFF7DEFF10BD03000220002936
:109AB00006D0002B04D0052200200A701B784B70C2
:109AC000704703000220002B08D0002906D05B78E5
:109AD00000200B70013B082B00D9183070470300A1
:109AE00010B50220002909D0002B07D00622481CFF
:109AF0000A7019000A3202F013F9002010BD10B5E7
:109B0000FFF7B0FF10BD02000B00022010B50029C6
:109B10000ED0002A0CD007211970118859701188B5
:109B2000090A997011180822D81C02F0F9F80020CF
:109B300010BD03000A00022010B5002B0CD0002934
:109B40000AD099785878090201431180901CD91CD9
:109B5000082202F0E5F8002010BD030010B5022035
:109B6000002909D0002B07D00822481C0A701900D0
:109B7000921802F0D5F8002010BD02000B00022060
:109B800010B500290BD0002A09D0092119701178CD
:109B900018185970511C062202F0C2F8002010BD9E
:109BA00010B5FFF75FFF10BD02000B00022010B5DB
:109BB000002A09D0002907D05178197011180622FF
:109BC000581C02F0ADF8002010BD030010B50220B3
:109BD000002909D0002B07D00A22481C0A7019005E
:109BE000063202F09DF8002010BD10B5FFF73AFFD5
:109BF00010BD02000B00022010B5002A06D000297B
:109C000004D018005178FFF753FB002010BDF0B5C9
:109C100085B017001E006A460623050008009181E2
:109C20009380FEF7C0FC1324011E02900CD0380074
:109C3000B047041E05D1280001A9FEF76FFA041EE3
:109C400002D0029802F02CF82800FFF701FA200059
:109C500005B0F0BDF0B504008BB0019115000021F6
:109C6000102202A801F0BCFE334EA700B85900280C
:109C70003CD0C388A34239D10378002B36D1427837
:109C8000062A18D102000100553235310C3006ABDE
:109C9000FFF7A9FA002829D12000FFF72FFE0200C4
:109CA00006A902A802F03CF8200002A901F080FFFA
:109CB00001200BB0F0BD816E002917D00B8A112A4C
:109CC00028D19D420ED101981231093A01F000FFCE
:109CD000012807D1BB5920009D6EFFF70FFE290018
:109CE0000200DEE732212000FFF7D8FC2000FEF75B
:109CF00001FF061E1BD0416A002918D00B8AAB4217
:109D000015D108220198123101F0E2FE01280ED18E
:109D1000716A0AE09D42E9D108220198123101F0EE
:109D2000D7FE0128E2D1BB59996E8A7EB9E720009F
:109D300001F01EFEBCE7C046FC68FF1FF0B56B4D8E
:109D400087007E5985B0337802900393002B00D0B2
:109D500087E0B368346A01937078062817D101222E
:109D60001B7D134202D0217B114218D102221342E3
:109D700002D0217B114251D10422134203D0237B14
:109D8000134200D08BE0019B5A7DEB5991E00738DC
:109D90000428F8D801F04CFD032E42678300B36E0F
:109DA000002B03D11C2001F03BFFB066EB599C6EE9
:109DB000002C1CD010220021200001F011FE02987E
:109DC000FFF79CFD01002000FFF72DFA02F000F8DC
:109DD0002082200008211230FFF725FA0298FFF7B1
:109DE0008DFDA076EB592100D888FFF70FFC0822E3
:109DF000EB591CE0B36E002B05D01A00198AF088CD
:109E00001232FFF70DFC0222019B197DEB59114222
:109E10003DD0207B10423AD0073208E0F488FCF7AE
:109E2000DBFD01002000FFF711FC0A22EB595A70FC
:109E3000029B9C002A595378073B042B11D8D088E9
:109E4000FEF758FE00284ED0C3895A08D218284978
:109E5000029B0298CB542B5941180433254801F03A
:109E60009FFD05B0F0BDFCF79FFD0300012083427C
:109E700001D100200393EB59DE88FCF79BFD039989
:109E800002003000FFF7ECFB019AEB59117D042230
:109E900011420CD0217B114209D00B22C7E7F68872
:109EA000FCF73CFD01003000FFF7EEFB6BE7019A89
:109EB000527D01210A4204D0607B084201D00C226D
:109EC000B5E702210A4204D0607B084201D00E228D
:109ED000ADE704210A4204D0627B0A4201D010227D
:109EE000A5E71222A3E7FA225200B0E7FC68FF1FA1
:109EF0000069FF1FB3A2001110B5064B1A780423A6
:109F0000100018401A4200D00348FFF727FA00203B
:109F100010BDC0468967FF1F1046FF1F70B50400C3
:109F2000FFF7D4FA051E43D12000FFF77FFA234E36
:109F3000A400A0598268937CDB0708D50321036A3B
:109F40001B790B40012B02D1017F0B430377431D8B
:109F5000D97F8B1E022B0DD8022900D00121C08889
:109F6000FCF790FF042133591A7F59700A431A777E
:109F7000280070BD01290CD102231022437000215A
:109F80000C3001F02DFD305910213530FFF74BF921
:109F9000EEE70529ECD10223D118437010220C30D2
:109FA00001F0BEFE04233259117F0B431377EAE719
:109FB00008251828DCD1053DDAE7C046FC68FF1FFC
:109FC000F0B58BB0059143887E4F9E00F459150083
:109FD0000493002C15D1012902D000200BB0F0BD54
:109FE000101D57781678FFF757F9EB683200029387
:109FF0002B7A0499019300903B002000FCF70CFFA2
:10A00000EBE7E388049A934201D00820E6E723783F
:10A01000012B00D1D4E0059B581E092800D9CFE0C0
:10A0200001F006FC05CE0A29CC506C859AB22900B5
:10A030000498FFF773FFD1E7200029001022453074
:10A0400001F06EFEB9594B78042B02D1013B4B70E5
:10A05000C3E70B000A00253335320C310498FFF7B3
:10A0600095F90498FFF702FA0522431E9841BB595F
:10A07000C0005A70B2E7200029001022553001F0CC
:10A080004FFE049B4F4C9D00295904980A0006ABD3
:10A0900055320C31FFF77AF929591022453106A8BB
:10A0A00001F016FD012808D10498FFF7F7F9059093
:10A0B000002804D106222B595A7005988EE70823F0
:10A0C0000593FAE763780C2B7AD1E36E002B03D16A
:10A0D0001C2001F0A5FDE066BB59D86E00286FD0AA
:10A0E0001022290001F01CFEBB590498DC6EFFF71A
:10A0F00005FC0D22A076BB595A706EE7E06E002871
:10A100005ED063780D2B5BD12B8808220382A91CBB
:10A11000123001F005FEBB599A68517D02221142AE
:10A1200026D0186A407B104222D00C32E4E76378D4
:10A130000E2B45D1236F002B03D1162001F070FDAB
:10A140002067BB59186F002803D01022290001F0A6
:10A15000E7FD0F22BB59CFE763780F2B30D1206F7B
:10A160000622691C103001F0DBFDBB599A68517D55
:10A170000422114203D0196A497B1142D5D1002132
:10A180000498FFF78BFA28E7636F002B0DD0BB59BB
:10A19000586F0028F3D01022290001F0C1FD0122E0
:10A1A000BB5952425B6F1A61E9E7142001F038FD98
:10A1B000BB5960675B6F002BE9D126E72978DFE7A1
:10A1C00007200BE7FC68FF1F10B5064C207001F05C
:10A1D0003FFC06212078FDF791FF0348FEF778FC4D
:10A1E00010BDC0460F69FF1F6993001100200BB21C
:10A1F00070B50D00834216DA264B187801F080FD09
:10A20000041E0DD00378922B0ED0A02B37D0224BFA
:10A210001878FF283AD0210001F0BAFD002835D186
:10A2200080200002684070BD43780E2B0BD03E2B7F
:10A23000EDD18378052B12D0082BE8D18179808865
:10A24000FFF7D8FA08E0154B82889A42DFD183687D
:10A250001878591CFEF7C0FE002817D1D7E7104B1D
:10A260001B785B0712D50F4B1B68002B0ED09B6829
:10A27000002B0BD0C289811D80889847ECE7FFF73F
:10A2800041FAA068002801D001F00AFD200001F089
:10A29000EFFCC5E70F69FF1F0946FF1F18200000EC
:10A2A0008967FF1FF868FF1F10B50078FFF712FAE3
:10A2B00010BD10B50078FFF7FDFA10BD0C23434325
:10A2C000084A10B59B185A68002A03D0012901D109
:10A2D000904710BD9B68002BFBD00029F9D198470F
:10A2E000F7E7C0462C69FF1F01238340094A10B5D8
:10A2F000946B1C439463506B98435063D46B200061
:10A300009843012901D120001843D063116B0B43FE
:10A31000136310BD00800040F0B500240127154BE9
:10A3200085B0DA6B144E03921A6C0192DA64019BC9
:10A33000E3403B4217D0039DE5403D400295E5B226
:10A3400002992800FFF7BAFF316A736A002908D022
:10A350003900002B01D0029979402800FFF7C4FF93
:10A3600001E0002BF9D101340C36172CDFD105B0F8
:10A37000F0BDC046008000401069FF1F064B012160
:10A380005A68C2400A4204D01B68C3401800084003
:10A3900070471B6DF9E7C046008000400122064B64
:10A3A0008240002903D0D9680A43DA607047D9682F
:10A3B0009143D960FAE7C0460038004030B5032425
:10A3C00044430F4BE25C1B199C785D7801232D1BE5
:10A3D0000135AB40013BA340A140DB430C001228F8
:10A3E00007D808499200521811681940214311609A
:10A3F00030BD054A11680B4023431360F8E7C0469F
:10A4000023C1001108F0004014F00040C21F70B5D5
:10A41000D4B20623092C0BD80125084C95400029FD
:10A4200008D00021FFF7CAFF23682B4323600023D5
:10A43000180070BD2368AB43F8E7C0460038004001
:10A44000214BF0B51B185B78022B21D10324444328
:10A450001E4A1F4EA35C12199478012215008540F4
:10A46000B76B013CE4B23D43A240B563194C1228DE
:10A4700015D89B0000290CD117495B1899680A432D
:10A480009A600123205C154A834011680B431360D6
:10A49000F0BD11495B18996891439960F1E70E4B43
:10A4A00000290DD159690A435A61225C1328E8D06A
:10A4B0000123203A93400A49086803430B60E7E709
:10A4C000596991435961F0E71069FF1F23C10011D9
:10A4D0000080004068C1001100F00040A0F0004082
:10A4E000A4F00040F8B500241B4E1C4D1C4B1B5D16
:10A4F000012B1FD1194A9269E2401A420BD0012266
:10A50000B25693402200143AD2B2022A09D8154911
:10A510004A6913434B61013402360C35172CE5D1DF
:10A52000F8BD0022B2560F499200521891680B43B1
:10A530009360F0E7022BEED1E7B23800FFF71EFF81
:10A5400001235840C1B23800FFF77AFF3800FFF707
:10A5500015FF6877DFE7C046F5C000111069FF1FDF
:10A560001169FF1F00F00040012202388240054BB4
:10A57000002903D059690A435A61704759699143C8
:10A580005961FAE700380040F8B50E0001210F00CC
:10A590008740114A0400D368FD43BB43D360831E48
:10A5A0008B4201D8FFF7E0FF00212000FFF72EFFCC
:10A5B0000A4A0B4B5168012E05D139431B195160D2
:10A5C0005E700020F8BD2940516002221C196270A3
:10A5D0009A6915409D61F4E7003800400080004012
:10A5E0001069FF1F012210B58240074B002906D0D9
:10A5F00019680A431A600121FFF7C6FF10BD1968E8
:10A6000091431960F7E7C046008000400C2370B505
:10A61000002543430A4A29009B181D70094B04007A
:10A620001B185D70FFF7B0FF0123A3400649280007
:10A630000A681A430A6005490A689A430A6070BDAD
:10A640002C69FF1F1069FF1F3480004030800040DC
:10A6500070B504000E00FF2813D003250540FFF756
:10A66000D5FF084AA3089B009B183F22ED00AA4093
:10A67000AE40196820009143314319600121FFF772
:10A680008DFE70BD18380040F8B50C244443134BC0
:10A690000500E4186368002B03D1A3681220002B87
:10A6A0001AD0022201270E4B00215B195A70280094
:10A6B0002770FFF769FF63681E1E08D0A3683E007D
:10A6C000002B04D02800FFF759FE4640F6B22800C0
:10A6D0003100FFF709FE0020F8BDC0462C69FF1FBE
:10A6E0001069FF1FF7B5C420FF222B4B80001958BB
:10A6F000002491433F3A0A431A508022274F5202C6
:10A70000274E1A60274B1D5D002D21D0A31E012B63
:10A7100003D80121E0B2FFF727FF012D18D11F4B0D
:10A720009B69E3402B4213D0E3B218000193FFF77B
:10A7300025FE01000198FFF755FFE3B2143B022B01
:10A740001DD801217156184A8D405369AB4353619E
:10A750003B7F002B0DD0E5B22800FFF795FF2800C6
:10A76000FFF70CFE7B7F0100834202D02800FFF739
:10A77000A5FD01340C370236172CC3D1F7BD0121DA
:10A7800000237156F3568D40074A9B009B189A6828
:10A79000AA439A60DCE7C04600E100E01069FF1FB1
:10A7A000F5C000111169FF1F00F0004070B50E00E8
:10A7B00015000400FFF72AFF0C236343094A200019
:10A7C0009B189D605E60FFF75FFFF021064B074A14
:10A7D0008900051E5A5002D02000FFF717FF2800FD
:10A7E00070BDC0462C69FF1F0000FF1F19A3001198
:10A7F00070B5134D07202C78002C1FD19822210012
:10A800005200280001F02CF90123C420FF222B70F4
:10A810000C4B80001C635C630B4B1C605C600B4B3F
:10A82000195891433F3A0A431A50802252021A6043
:10A830000D20074A074901F033F8200070BDC046DB
:10A840001069FF1F00800040A0F0004000E100E020
:10A85000E5A60011E5A40011030010B50620072BA2
:10A8600009D8054A137000F0BBFFD7210020034B25
:10A87000034A89005A5010BD3846FF1F0000FF1FD1
:10A88000151BFF1F70B51D0002240C2910D8094AA2
:10A89000CA40D2070CD5FBF741FF041E08D1059A28
:10A8A00004992800FBF756FFFCF7C4FDFFF724FBD3
:10A8B000200070BD1210000030B50D7802232C006E
:10A8C0009C43184201D02B431C0008252300AB43B6
:10A8D000284201D02B00234320241D00A543204201
:10A8E00001D01C4325002A230D70184204D0117892
:10A8F0001E3B0B43137030BD0028FCD10C21137894
:10A900008B43F7E7F8B51D0006AB1B88140007AAB8
:10A910000E000B201778002B27D10A78022A49D184
:10A920004A68507811780002244A084380180428A5
:10A9300040D800F07DFF03121D1B2300F06801F0DA
:10A94000B7F9021CC0B2B84200D93A1CD2B22000FA
:10A95000F1682A8001F0E4F906E00222F3681B881E
:10A960002A8023701B0A63700020F8BD0622EEE7E0
:10A9700001232B80F3681B782370F5E7F368002B25
:10A9800016D008222A801A8822701A88120A627049
:10A990005A88A2705A88120AE2709A8822719A889C
:10A9A000120A6271DA88A271DB881B0AE371DBE7A5
:10A9B0002B80D9E701202B80D7E7C04600D6FFFFC8
:10A9C000F7B516000A781D0008AB1F880C0001239C
:10A9D000022A18D14A685078117800022B4A08439D
:10A9E000801803280FD800F023FF02254439E068BF
:10A9F00001F05EF9C0B20723B84204D37B1901937A
:10AA0000152B02DD0D231800FEBDE0682A00310081
:10AA1000C01901F085F96B4600209B88E268D0548C
:10AA20001B4B1B68834203D01B68834200D09847AE
:10AA30000023E8E70B23002FE5D1022DE2D1737844
:10AA400032781B021343E2681380114B1B68002B02
:10AA5000EED01B68002BEBD00120E8E70B23002F82
:10AA6000D1D1062DCED12A003100E06801F058F98D
:10AA7000DEE70B23002FC6D1012DC3D13278753309
:10AA8000012AC0D8E3681A70D2E7C04600D6FFFF9B
:10AA90001C6BFF1F70B50C001500072837D800F09D
:10AAA000C7FE041436361B36242E182015290BD861
:10AAB000184E16220021300000F092FF22002900DB
:10AAC000300001F02DF9002070BD18200229FBD1C3
:10AAD0001288114B1A80F6E718200829F4D10A00D1
:10AAE0000E48290001F04CF8EDE718200129EBD1C0
:10AAF0000B4B10780B49DA69FFF7DEFEE3E718200D
:10AB00000129E1D1064B10780749DA6BF4E70220FE
:10AB1000DAE7C046046BFF1FB646FF1FAC46FF1FB7
:10AB20003C46FF1F6446FF1F8446FF1F030010B50D
:10AB30000020DB0704D50721024A034800F08CF807
:10AB400010BDC04680C100113C46FF1F054A0300EE
:10AB50001068002803D082889A4201D1806870472B
:10AB60000068F6E7206DFF1F0A88030008009A427C
:10AB700004D08A8804309A4200D000207047000038
:10AB8000F8B5F82200230D4F0D4E796805004243B9
:10AB90003370994200D07B600A4C0021200000F005
:10ABA0001FFF00231A007C60AB4202D100203370EB
:10ABB000F8BD01332280DBB2F834F5E7206EFF1FC9
:10ABC0001C6EFF1F246DFF1F73B56B4601900600BE
:10ABD000684615001980FCF75FFF041E11D1002D97
:10ABE0000FD07689002E11D00C2001F019F8002822
:10ABF0000ED0084A0460136886808560002B02D15D
:10AC00001060200076BD1A001B68F7E70224F8E701
:10AC10001324F6E7206DFF1F012100220A4B10B517
:10AC200049420A4C198099809A719A70084B207099
:10AC3000012019805A60FFF7A3FF2078FCF78AFFF4
:10AC40000448FDF745FF10BD246BFF1F286EFF1F52
:10AC5000206EFF1F05AD0011022310B5002802D0A1
:10AC6000FFF7B2FF0300180010BD0000030010B58D
:10AC70000020DB0704D50421024A0348FFF7A4FFA4
:10AC800010BDC04694C10011BC46FF1FF0B50E2692
:10AC900087B003930CAB1F8802ABF61805000800C1
:10ACA00031000292FDF77AF804000120002C0FD049
:10ACB0003088FFF74BFF03000E20002B08D05E68A2
:10ACC000002E05D021002800039B029A0097B04770
:10ACD00007B0F0BD0A4B10B5984207D101220023FE
:10ACE00052420A808B708A808B7110BDFFF73CFF47
:10ACF0000028FAD001235B42038000238370F4E72D
:10AD0000FFFF0000F8B5050001290AD1134E002409
:10AD10003388F827AB4219D028001149FFF7DAFF32
:10AD200006E0022904D10139FDF750FF0028EDD0DB
:10AD3000F8BD3B0063437268D018D35A002B09D08A
:10AD40003A00002100F04CFE0134E4B2054B1B78C0
:10AD5000A342EED801235B423380DDE7206EFF1F64
:10AD6000246BFF1F1C6EFF1F10B5FFF7FDFE0300D5
:10AD70000020834200D0987810BD0000F0B589B063
:10AD80001C000EAB80CB03901E8810AB1B78049286
:10AD900002930B7A0D00DB0616D42B780593022B59
:10ADA00024D00498FFF7D2FE002812D003689C46F6
:10ADB000002B0ED0029B2200019329003B00644629
:10ADC00003980096A04705E00498FFF7BFFE00280F
:10ADD00002D10E2009B0F0BD8368002BF9D00A2201
:10ADE0002900039898470028D7D0F3E76B68587874
:10ADF0001A786B4B000210439842D2D8043B984219
:10AE000010D2684B984242D015D8674BC018012821
:10AE1000C7D80B20002EDDD1EB681A7859683A802C
:10AE2000200028E0614BC018032800D979E000F029
:10AE3000FFFC846A789E5E4B9842B2D10B20002EB4
:10AE4000C8D101233B80EB6831001B7823706889EF
:10AE5000013080B2FCF7A2FF3A88031E0ED00178C1
:10AE600002328A183A80428962704289120AA270BC
:10AE700059680278E01C00F053FF06E004323A8083
:10AE800031000422601C00F0ABFD0020A2E70B2083
:10AE9000002E9FD1EB6807A91E8804233B80330A4C
:10AEA000300026706370FCF779FF051E28D004ABD4
:10AEB0009A890E2304A95B183E49C668FCF7E2FF95
:10AEC00000280BD12B783C486A680599FBF798FB62
:10AED000002803D1012304AA5B42D3813278022ADD
:10AEE00006D17168201D00F01BFF3B8802333B80B8
:10AEF0000E2304AA9B181B88A3701B0AE370C4E7E7
:10AF000004ABDE81F4E70B20002E00D062E7E96895
:10AF10000398FFF729FF02233B802070000A60702E
:10AF2000B3E70B20002E00D054E70222EB681B8809
:10AF30003A8023701B0A6370A7E7E86800F0B8FE48
:10AF4000C2B203000720B24200D243E70DD00299FB
:10AF5000DBB27118994202DB921BD3B20293029BBF
:10AF6000E9681A003B8089195AE70023F6E70B20AD
:10AF7000002E00D02EE70722EB683A801A78227064
:10AF80005A7862705A88A2705A88120AE2701A7946
:10AF90002271DA886271DB881B0AA37175E7C046EB
:10AFA000042900000228000000D8FFFFFFD6FFFFA1
:10AFB00003280000FFFF0000C4C00011F0B58DB0F1
:10AFC0006B460020089120229B5E83423DDAA64B0F
:10AFD000187800F095FE071E32D00378B02B2CD1E4
:10AFE0000079023816281FD800F002FD17001E0055
:10AFF0001E001E0031001E0096001E001D011E00D6
:10B0000052011E0073011E00CD011E0050021E00E1
:10B010001E001E008E021E00E302944B94491B8802
:10B0200078880B80FBF72CF83800FCF7ADFF914BCC
:10B030001B68002B01D038009847380000F018FE3C
:10B040008020089B0002434018000DB0F0BDF6229E
:10B050000021874800F0C4FC0BAA3B7B7989388922
:10B0600000923A000D32FCF7B1FD0400804B1B78D2
:10B07000002C3FD146E0804B788805937F4B410000
:10B08000CB5A0BAE073BDBB232880293002301930D
:10B090007B4B210006930093059BFFF76FFE744DD9
:10B0A000002810D1069B3A8A1B889A420BD138009F
:10B0B0000599123000F00CFD002804D02B7862892D
:10B0C0009B00EB185A80162306A81B183288200014
:10B0D0007989FCF7D7FE2B7804009A00AA185188CA
:10B0E0000029C3D00133DBB22B70002807D006A99A
:10B0F000C98A9180634A12889A42BCD802E0012131
:10B1000049429180002B04D059497888FAF7ECFF26
:10B110008AE73E890A2479E000253E89574B069349
:10B120007B88069A5B009B5A033B9D4202DB002D05
:10B13000F0D05BE0162206A812183B7B79890092BA
:10B140003A0030000D32FCF741FD0590002858D040
:10B150004689017A7888FCF703FD041E44D1464BEA
:10B1600078880793069B4100C95A454B0439C9B2F8
:10B1700006AAD28A06930291019400930599079B2F
:10B18000FFF7FCFD041E2FD1069B39491A88931C3A
:10B19000002D26D14B807988384B4900CB5A511964
:10B1A000033B8B4220DD059B31485B8941190B71C4
:10B1B000A91C0135C9B2EDB2059145191B0A2B71C5
:10B1C000059B2D490433181800F0AAFD2C4B059A55
:10B1D0001B88D318DDB22C4B9E4205D00136B6B287
:10B1E0009CE749889942D6D0002D0CD0204C2800ED
:10B1F000618800F045FB207021007888FAF784FF11
:10B2000012E7059CF0E7002C00D183E77B78142B34
:10B2100000D109E716493B794E800B700C71788894
:10B22000FAF724FF00E7162406ABE418210038895A
:10B23000FCF7B4FD011E00D1B7E1788822880F4CDD
:10B2400045002C5B0A4D013CE4B2029400240F4BF4
:10B2500001940095FFF792FD041E00D014E129002F
:10B260007888FAF761FFDFE6286EFF1FA845FF1F09
:10B270002C6BFF1F206BFF1F266CFF1F5C67FF1FDF
:10B280001C6DFF1FA645FF1FFFFF00002E6BFF1F59
:10B29000162406ABE41821003889FCF77FFD011E57
:10B2A00000D182E178882288AE4C45002C5BAE4DFF
:10B2B000013CE4B202947C89AC4B01940095FFF709
:10B2C0005DFD041E00D0DFE029007888FAF736FF24
:10B2D000AAE60025A44B1D803B00FE331B78A24A42
:10B2E00078880792AB4208D99E4B1288069306993C
:10B2F00043005B5A013B9A4203DB0799FAF728FFA8
:10B3000092E616246B00FB18059306ABE418059B28
:10B3100021001889FCF742FD011E03D1059B012481
:10B320001E8973E77888924B2288069C0993430014
:10B330001B5B904E013BDBB202930023009601930E
:10B34000099BFFF71BFD041E02D0059B1E895DE7CC
:10B350007B88069A5B009B5A079A108832881218DD
:10B36000934202DC1B1A013B33807F4C023032884F
:10B370000999001900F0D4FC2388328801359B1804
:10B380002380EDB2A8E70BAA3B7B7989388900922C
:10B390003A000D32FCF71AFC00250590059B002BA6
:10B3A00004D10A24002D00D16EE060E0059B78886E
:10B3B000197AFCF7D5FB0100041E63D1694C6C4B74
:10B3C000788806940993069B4400E45A694B063C2E
:10B3D000E4B20BAE32880793029401910093059971
:10B3E000099BFFF7CBFC041E4CD1079B5E491B88D1
:10B3F0001A1D002D30D14A80059B5B4C5A89631978
:10B400001A716B1C9BB2E318120A1A71162306A854
:10B4100032881B1879890598FCF734FDFF21AA1C96
:10B420002E1D03350B00059092B2B6B2ADB20028C6
:10B4300003D006ABDB8AD9B21B0AA21865191171B9
:10B440002B714C4D301D2A884949201800F068FCAA
:10B450002B88F618B5B2A1E74988914207D17A88BE
:10B4600006995200525AEB18053A9A42C4DC3E4CF7
:10B470002800618800F0ACFA207021007888FAF783
:10B4800071FED1E5002DF2D13E89BFE6162606AB4E
:10B49000F61831003889FCF781FC3D000400FF35C7
:10B4A00000282DD0037A9B060CD400227B89398991
:10B4B000788800923A000C32FFF7E8FB041E10D0A7
:10B4C0003E8915E03088FFF741FB00281AD08368D9
:10B4D000002B17D02100122278889847041EE4D050
:10B4E000EEE7AB78002B02D17888FAF74BFE002606
:10B4F000AB78002B00D097E5002C00D194E585E6D1
:10B500000124DDE70E24DBE7162506ABED18290044
:10B510003889FCF743FC041E47D0037A9B0611D4FC
:10B52000154A7B881188994203D01448814207D17B
:10B530001380134BF8261D780023D9B2A94221D3DA
:10B540000924A1E72888FFF701FB00282FD0836892
:10B55000002B2CD02100122278889847041EDFD0BF
:10B5600092E7C0465C67FF1F2C6BFF1F2E6BFF1F0F
:10B57000266CFF1F1C6DFF1F206EFF1FFFFF0000CA
:10B580001C6EFF1F31005943546801336018615A23
:10B590000029D2D13C0008342100F82200F0C0FB81
:10B5A00021007888FAF7F6FD3EE501246CE70E24C9
:10B5B0006AE71D4B1A887B889A4231D07888FAF75F
:10B5C000F3FD31E5F823059851684343CD18C95A76
:10B5D00000291FD03B7A012B0BD16C88AB8878886F
:10B5E000AA1D0094FFF752FB041E02D000233B72F9
:10B5F0002E88F8220021280000F0F2F900232B8089
:10B60000059B0133DBB20593084B05991B78064A6D
:10B610008B42D7D801235B421380002CCED0F5E5B6
:10B62000002634000596EFE7206EFF1F1C6EFF1FFB
:10B6300070B504000E001500FFF796FA031E08D13E
:10B6400031000548FFF790FA03001120002B02D0CB
:10B650001C8000209D7070BDFFFF0000F8B50B4FEF
:10B6600006003B780D001400FF2B0ED00A2000F0DE
:10B6700037FB011E09D0B1230380002346800371EC
:10B68000C5800481387800F083FBF8BDFD46FF1FBC
:10B69000F7B50F0008A90600088809A90B24098836
:10B6A000002821D10234022B1ED1557813782D02A7
:10B6B0001D432B008B4301937334002B14D1FB6883
:10B6C000300019000093FFF74FFB019C85420BD01F
:10B6D0002A0030000099FFF7ABFF041E04D12A00B6
:10B6E00030007989FFF7BAFF2000FEBDF0B50E7873
:10B6F00085B003900AA805880120022E0DD14C6860
:10B700002778647824023C43054FBC4205D1039856
:10B71000DBB201960095FFF7BBFF05B0F0BDC04658
:10B720000229000010B504000C4800F081F90C4813
:10B73000A16B00F07DF90B48E16B00F079F90A4844
:10B74000216C00F075F9094B0948196800F070F98F
:10B75000084B1B68002B00D09847FEE776BF00110E
:10B760008CBF00119BBF0011AABF001104ED00E0C7
:10B77000B9BF00112C6EFF1F002307B501A801936C
:10B78000FFF7D0FF044A0548002110B5121A00F057
:10B7900027F9F8F715F9FEE7306EFF1F0047FF1F86
:10B7A00001B40248844601BC604700BF6D30FF1FF2
:10B7B00001B40248844601BC604700BFB54C01009B
:10B7C00001B40248844601BC604700BFC53F000089
:10B7D00001B40248844601BC604700BFB14E00007E
:10B7E00001B40248844601BC604700BF151BFF1F1F
:10B7F00001B40248844601BC604700BF2124000018
:10B8000001B40248844601BC604700BFC534FF1F35
:10B8100001B40248844601BC604700BF55220000C5
:10B8200001B40248844601BC604700BFE139FF1FF4
:10B8300001B40248844601BC604700BFC53DFF1FFC
:10B8400001B40248844601BC604700BF613BFF1F52
:10B8500001B40248844601BC604700BF156B01007B
:10B8600001B40248844601BC604700BF25260000A1
:10B8700001B40248844601BC604700BF691F000054
:10B8800001B40248844601BC604700BF350E000089
:10B8900001B40248844601BC604700BF4D1F000050
:10B8A00001B40248844601BC604700BFE532FF1F77
:10B8B00001B40248844601BC604700BF893CFF1FB9
:10B8C00001B40248844601BC604700BFE92800007B
:10B8D00001B40248844601BC604700BF5D17000008
:10B8E00001B40248844601BC604700BFB53CFF1F5D
:10B8F00001B40248844601BC604700BF5D38FF1FA9
:10B9000001B40248844601BC604700BFEDA50000B9
:10B9100001B40248844601BC604700BF2D38FF1FB8
:10B9200001B40248844601BC604700BF017F0000AB
:10B9300001B40248844601BC604700BF055E0000B8
:10B9400001B40248844601BC604700BF851F000067
:10B9500001B40248844601BC604700BF5118FF1F74
:10B9600001B40248844601BC604700BF056A00007C
:10B9700001B40248844601BC604700BF091B0000B7
:10B9800001B40248844601BC604700BFB930FF1FC4
:10B9900001B40248844601BC604700BF8D1200001C
:10B9A00001B40248844601BC604700BFA9460100BB
:10B9B00001B40248844601BC604700BF0189000011
:10B9C00001B40248844601BC604700BFED4A010053
:10B9D00001B40248844601BC604700BF090E000064
:10B9E00001B40248844601BC604700BF154D010008
:10B9F00001B40248844601BC604700BFD93DFF1F27
:10BA000001B40248844601BC604700BF8B5201006C
:10BA100001B40248844601BC604700BFA13BFF1F40
:10BA200001B40248844601BC604700BFA54F010035
:10BA300001B40248844601BC604700BFE53A0100FA
:10BA400001B40248844601BC604700BFC521000024
:10BA500001B40248844601BC604700BFC92600000B
:10BA600001B40248844601BC604700BFB70E000025
:10BA700001B40248844601BC604700BF6DBC0000B1
:10BA800001B40248844601BC604700BFC94A0100B6
:10BA900001B40248844601BC604700BF3555000030
:10BAA00001B40248844601BC604700BF4532FF1F15
:10BAB00001B40248844601BC604700BF0D5201003A
:10BAC00001B40248844601BC604700BF3D18000035
:10BAD00001B40248844601BC604700BFCD4C010060
:10BAE00001B40248844601BC604700BFDD66010026
:10BAF00001B40248844601BC604700BF2D39FF1FD6
:10BB000001B40248844601BC604700BF1D4B0100E0
:10BB100001B40248844601BC604700BF9DA90000F3
:10BB200001B40248844601BC604700BF291C0000E4
:10BB300001B40248844601BC604700BFE93AFF1FD8
:10BB400001B40248844601BC604700BF4551010072
:10BB500001B40248844601BC604700BF5D32FF1F4C
:10BB600001B40248844601BC604700BFC95C0100C3
:10BB700001B40248844601BC604700BF3938FF1F4A
:10BB800001B40248844601BC604700BF810E00003A
:10BB900001B40248844601BC604700BF4550000024
:10BBA00001B40248844601BC604700BF65710100D2
:10BBB00001B40248844601BC604700BF311B00004D
:10BBC00001B40248844601BC604700BF456B0100D8
:10BBD00001B40248844601BC604700BF1147010020
:10BBE00001B40248844601BC604700BF213BFF1FEF
:10BBF00001B40248844601BC604700BFF535FF1F11
:10BC000001B40248844601BC604700BFB352010042
:10BC100001B40248844601BC604700BF8552010060
:10BC200001B40248844601BC604700BF3D4B01009F
:10BC300001B40248844601BC604700BFC51D000036
:10BC400001B40248844601BC604700BF350E0000C5
:10BC500001B40248844601BC604700BF5549010059
:10BC600001B40248844601BC604700BF090E0000D1
:10BC700001B40248844601BC604700BF434D010047
:10BC800001B40248844601BC604700BFADAE00006D
:10BC900001B40248844601BC604700BF7918000027
:10BCA00001B40248844601BC604700BFD949010085
:10BCB00001B40248844601BC604700BFDD52010068
:10BCC00001B40248844601BC604700BF9D32FF1F9B
:10BCD00001B40248844601BC604700BF014C01002A
:10BCE00001B40248844601BC604700BF1D4D0100FD
:10BCF00001B40248844601BC604700BFF30E000057
:10BD000001B40248844601BC604700BFF54E010003
:10BD100001B40248844601BC604700BF8534FF1F60
:10BD200001B40248844601BC604700BFE94C0100F1
:10BD300001B40248844601BC604700BF75A90000F9
:10BD400001B40248844601BC604700BFB13DFF1FFB
:10BD500001B40248844601BC604700BFE5480000CA
:10BD600001B40248844601BC604700BF7D18FF1F34
:10BD700001B40248844601BC604700BF514701003E
:10BD800001B40248844601BC604700BF0D3CFF1F60
:10BD900001B40248844601BC604700BF594F01000E
:10BDA00001B40248844601BC604700BFE1170000AF
:10BDB00001B40248844601BC604700BFC9A9000025
:10BDC00001B40248844601BC604700BFC56D010054
:10BDD00001B40248844601BC604700BF29510100FC
:10BDE00001B40248844601BC604700BF59520100BB
:10BDF00001B40248844601BC604700BFD91B000063
:10BE000001B40248844601BC604700BF0124000021
:10BE100001B40248844601BC604700BF51250000C0
:10BE200001B40248844601BC604700BFD53AFF1FF9
:10BE300001B40248844601BC604700BFF94C0100D0
:10BE400000030102020303030403050006020700C6
:10BE5000080209030A030B030C000D000E030F0375
:10BE6000100311031203130314031502160200003A
:10BE7000B53D0011E93D0011000000000200000086
:10BE800086BE0011192A0F1809000000F1590000A0
:10BE9000FD240000D9810011EDA1001141760011AF
:10BEA000DD7F0011B5540011BDAF00111D5100110F
:10BEB000A53F0011D540001100000000161600003B
:10BEC00002000000CCBE0011F4FFF3FFD2FC000022
:10BED0001542001100000000000000005475796157
:10BEE0000042312E33003030313700676974687595
:10BEF000622E636F6D2F7076767800544842310061
:10BF00000200000014BF0011292A282A272A262A05
:10BF1000252A242A0A180000E20400007102000009
:10BF200078EC0000744000001027000060F0000072
:10BF300006640000204E0000000000000500000024
:10BF40001F501D00023CB400000117001300000048
:10BF5000A1020000303132333435363738394142AE
:10BF600043444546005048592B36325858504C559A
:10BF70005330353034005B48617264206661756C03
:10BF8000742068616E646C65725D0A004C522020FA
:10BF9000203D203078253038780A0050432020207A
:10BFA0003D203078253038780A0050535220203D0B
:10BFB000203078253038780A0049435352203D20FC
:10BFC0003078253038780A00B95800110D59001121
:10BFD0000000000002000000E0BF00116F2A6E2A7E
:10BFE0001A18EAD8BC80F0FC6000000000000000D5
:10BFF00000005F066B2F363D7D077F3F777C596ED3
:10C000007971000001A00000000000006410B71D5D
:10C01000C8206E3BAC30D9269041DC76F4516B6B76
:10C020005861B24D3C7105502083B8ED44930FF038
:10C03000E8A3D6D68CB361CBB0C2649BD4D2D386EE
:10C0400078E20AA01CF2BDBDFB349B5F800000803B
:10C05000001000000000000043620011CD780011C4
:10C0600067620011D57C0011EB620011AB7C0011FE
:10C0700061630011817C0011B3630011497E0011DE
:10C080001B640011497E00114D640011037E0011F4
:10C0900061630011397C0011D9630011E17D001149
:10C0A0000000000000000000BF640011E17D0011ED
:10C0B00021650011E5780011052A042A012A002AC9
:10C0C0000229032801280028011800180000000098
:10C0D00000000000000000000000008701010201D4
:10C0E0000201010201020303040103010101010134
:10C0F0000303020103000D000E00100011001300E5
:10C100001401070108010A010B011C011D020402B0
:10C1100005020702080219021A021C021D0301038C
:10C12000020317000201000504000807000B0A00C3
:10C130001716001D1C010201010504010E0D01115D
:10C1400010011413011716011A19020201020B0A39
:10C15000020E0D0211100214130217160305040338
:10C160000807030B0A030E0D0001020307090A0B5F
:10C170000E0F101112141718191A1B1F202122005C
:10C1800005A90011C1A90011000000000200000073
:10C19000CAC0001100000000EDB600110000000050
:08C1A00002000000C8C00011FC
:020000041FFFDC
:1000000000000000113F00118CBE001188BE0011DD
:100010000C64FF1F00000000000000000000000052
:1000200000000000000000000000000000000000D0
:1000300000000000000000000000000000000000C0
:1000400000000000000000000000000000000000B0
:1000500000000000000000000000000000000000A0
:100060000000000000000000000000000000000090
:100070000000000000000000000000000000000080
:100080000000000000000000000000000000000070
:100090000000000000000000000000000000000060
:1000A0000000000000000000000000000000000050
:1000B0000000000000000000000000000000000040
:1000C0000000000000000000000000000000000030
:1000D0000000000000000000000000000000000020
:1000E0000000000000000000000000000000000010
:1000F0000000000000000000000000000000000000
:1001000000000000000000000000000000000000EF
:1001100000000000000000000000000000000000DF
:1001200000000000000000000000000000000000CF
:1001300000000000000000000000000000000000BF
:1001400000000000000000000000000000000000AF
:10015000000000000000000000000000000000009F
:10016000000000000000000000000000000000008F
:10017000000000000000000000000000000000007F
:10018000000000000000000000000000000000006F
:10019000E934FF1F3133FF1FC1660100000000007A
:1001A000000000000000000000000000000000004F
:1001B000000000000000000000000000000000003F
:1001C000000000000000000000000000000000002F
:1001D000000000000000000000000000000000001F
:1001E000000000000000000000000000000000000F
:1001F00000000000000000000000000000000000FF
:1002000000000000000000000000000000000000EE
:1002100000000000000000000000000000000000DE
:1002200000000000000000000000000000000000CE
:1002300000000000000000000000000000000000BE
:1002400000000000000000000000000000000000AE
:10025000000000000000000000000000000000009E
:10026000000000000000000000000000000000008E
:10027000000000000000000000000000000000007E
:10028000000000000000000000000000000000006E
:10029000000000000000000000000000000000005E
:1002A000000000000000000000000000000000004E
:1002B000000000000000000000000000000000003E
:1002C000000000000000000000000000000000002E
:1002D000000000000000000000000000000000001E
:1002E000000000000000000000000000000000000E
:1002F00000000000000000000000000000000000FE
:1003000000000000000000000000000000000000ED
:1003100000000000000000000000000000000000DD
:1003200000000000000000000000000000000000CD
:1003300000000000000000000000000000000000BD
:1003400000000000000000000000000000000000AD
:10035000000000000000000000000000000000009D
:10036000000000000000000000000000000000008D
:1003700079B700110000000000000000000000003C
:10038000000000000000000000000000000000006D
:10039000000000000000000000000000000000005D
:1003A000000000000000000000000000951AFF1F80
:1003B000000000000000000000000000000000003D
:1003C000000000000000000000000000000000002D
:1003D000000000000000000000000000000000001D
:1003E000000000000000000000000000000000000D
:1003F00000000000000000000000000000000000FD
:081838003072FF1F4118FF1F71
:10184000024981F3088802F0ABFB00003072FF1FF1
:1018500010B502F0D5FB072804D0122808D00228C2
:1018600008D010BD044A0420136B01331363F8E75A
:101870000220F6E71420F4E70468FF1FF8B507001C
:101880000C0026002500503630785135002804D150
:101890000300287058342370F8BD2978CA00481E08
:1018A0008141A3183800A25C5B68C9B2FFF7D0FF82
:1018B00000280DD12B78DA00A218013350602B706C
:1018C0003378044A013B3370136A01331362D8E75B
:1018D0000123DFE70468FF1F5C234343074910B57A
:1018E000C9180B0058331B78012B05D1FFF7C6FF31
:1018F000034A936A0133936210BDC0463868FF1FE4
:101900000468FF1F10B502F05BFB064A01211300BB
:1019100010CB4942D967044B136002F019FB200039
:1019200010BDC04600E100E01000100010B504003A
:1019300002F046FB024B1C6002F00AFB10BDC046E1
:1019400000E100E010B5040002F03AFB4021094A32
:10195000200013688B43136002F0E2FA01F0A6FD49
:101960000022054B01201A60044B04321A6002F079
:101970009FFAFEE71CF00040C4F00040C0F00040B9
:10198000431E5A425341A022F0B5D2015B4213409C
:10199000154D164A40019B182A18127E8BB00191F2
:1019A000002A1BD01A000832D46F0022E6B206AF1C
:1019B000E4B294420EDC2818C369002B08D00199C8
:1019C00002AA117106AA049202AA167303A89847E4
:1019D0000BB0F0BD1978B9540132EAE71A7D1A78D4
:1019E00006AB01261A70E6E7C46AFF1F00400040FC
:1019F000F0B5254B04004001C25C85B0002A2BD015
:101A00001A18117E002927D0917E002924D011793F
:101A1000022921D11689D788D168F51BADB22A1CBD
:101A2000102D00D9102292B2BE4217D118180123EE
:101A300003710023C269C38003819A4206D06846BD
:101A4000032103730171029301A890470820002C21
:101A500000D0192001F022FC05B0F0BD013C654228
:101A60006C41A0256442ED012C40084D1B186419FF
:101A7000074D0633013A92B2AA42EDD01888461CAF
:101A80001E80085C2070F5E7C46AFF1F004000401C
:101A9000FFFF00000F220E4B10B59868104002386F
:101AA0000A280BD802F08EF90D0A0B0A0A110A0A4D
:101AB0000A0A060002210020FFF762FF10BD012183
:101AC000F9E70020FFF794FFF8E7DB6FF6E7C04681
:101AD000004000400F220E4B10B5986810400238AD
:101AE0000A280BD802F06EF90E0A0B0A0A120A0A2B
:101AF0000A0A060002210120FFF742FF10BD012162
:101B00000800F9E70120FFF773FFF7E7DB6FF5E760
:101B10000090004013B5334C2378072B3DD8324B4F
:101B20001A78324B002A39D18022196852020A43AE
:101B30001A60252001F0F4FF20232D4A11680B4381
:101B4000802113606B460422C905086807331042E0
:101B500028D080210422C905C86810422ED08021D7
:101B60002020C905CA688243CA6014221A701A78F4
:101B7000002A2FD18021C905C86820320243CA60DB
:101B800014221A701A78002A28D11A4B1A7D22784A
:101B90005A601D221A705932DA6013BD1A6816494C
:101BA0000A40C5E7086802430A6014221A701A78CE
:101BB000002ACED01A78013AD2B2F7E7C8680243B9
:101BC000CA6014221A7019784A1ED2B21A700029FB
:101BD000F9D1C4E71A78013AD2B2C7E71A78013AC4
:101BE000D2B2CEE73846FF1F0047FF1F3CF000404F
:101BF0003046FF1F00200040FFFFFEFF564B70B530
:101C00001B68012B03D1554A936D0133936502F094
:101C10001FFA534B534A1860534B544C1A6001231C
:101C2000534A1360534A13602378002B06D00622D0
:101C30005149524802F0BCFA00232370504A514BDC
:101C400010681B78C1B2002B0ED14F4CC0B2237864
:101C50005BB2002B4FDB237824785BB264B21B04A9
:101C600024021B191B1813600B1C50294ED950233A
:101C7000464A47491078DBB2FF2202284BD1086858
:101C8000444C454D267890432A78964254D9227880
:101C900024782E78023B5D10A31B6B435201D31AAC
:101CA00010335B111843086002F052FA031F012B36
:101CB00045D83A4B1B78002B06D0394B1B78002BAC
:101CC00002D0002002F0C4FAA122364B920099788B
:101CD000354B4A431B689B18832292009B181B7844
:101CE000033B012B03D8AF20400002F039FA012258
:101CF0002E4BDA8270BD237824785BB264B2FF3356
:101D0000FF341B0424021B190138ABE7CAB2022AB4
:101D1000AED20223ACE70868254C264D26789043C6
:101D20002A78964208D9227824782D78023B5B10D5
:101D3000641B63435201B2E72378DBB2B2E70228A7
:101D4000D5D11D4B1B78013B022B03D91B4B1B78B4
:101D5000022BCCD16C20C8E79809FF1FFC0FFF1F96
:101D60003C67FF1FFF3F0000141003404067FF1F48
:101D70000C10034000100340D50BFF1F7211FF1F12
:101D8000B40003408C09FF1F680AFF1F490AFF1FA8
:101D900094000340460AFF1F470AFF1FF908FF1F70
:101DA0002209FF1F300DFF1F3409FF1FBC0BFF1F4F
:101DB000440AFF1F450AFF1F1C09FF1F2309FF1FBD
:101DC00010B502F095FA0022014B1A8010BDC046F2
:101DD0003867FF1F10B502F02BF8A121054A8900D2
:101DE0009478054A61431268044B5218528C1A8049
:101DF00010BDC046300DFF1F3409FF1F3867FF1F9D
:101E000010B50D4B0D4A9978A1239B004B431268E6
:101E1000D218531DD97F0A4B1B88994209D2441C02
:101E200007D0C82805D0D2695B1A5A43054B5343E3
:101E3000C01802F02DFA10BD300DFF1F3409FF1F2E
:101E40003867FF1F7102000070B5244D2B68002B0E
:101E500028D002F09DF92B68D8402B680400002B95
:101E600027D002F03DFA2B68D8401D4B1D4A9978C7
:101E7000A1239B004B431268D118D25C91239B0095
:101E8000002A20D0CA580132CA50174B17491B6884
:101E90000868834214D3D23B181A012A1AD0144B73
:101EA000186070BD02F074F9124B196801F0D0FF90
:101EB000D3E702F015FA0F4B196801F0C9FFD4E718
:101EC0000D495B18E8E7CA500C4B1B68DB68E41847
:101ED000201AE4E7F530FF30E1E7C0461C08FF1F99
:101EE000300DFF1F3409FF1F9C09FF1F3C67FF1FB8
:101EF000A009FF1F1808FF1F2DFF3F004467FF1FA9
:101F000070B504000D00282916D10300A433C2883F
:101F10001B889B1A0B4A9BB293420DD906006A3666
:101F200005223100653002F0C3F9002804D13100E8
:101F3000200002F0FDF870BD2900200002F050F8EA
:101F4000F9E7C046FE7F0000F8B50400012002F06A
:101F500097F902F055F9174A17491060174D030019
:101F6000886A174E28607568AC46164D2F680025A4
:101F7000BC4501D275687D1B134E00193560C862DF
:101F8000A4204C6A40032043486210490978002984
:101F900005D00F490978022902D10F3B1360F8BD23
:101FA000012901D1083BF9E7032901D1053BF5E7F8
:101FB000033BF3E7E408FF1F00F00040340AFF1F73
:101FC00028100040180AFF1F1C0AFF1F1C09FF1FD2
:101FD0004A0AFF1F70B580241025E405A3682B432F
:101FE000A36002F01DF9A368AB43A36070BD0000BD
:101FF000F7B5160080221C001023D20501919168CC
:1020000005000B43936000225A4BD7301A6001F051
:1020100017FF9D232A002F009B00EB58CA32012195
:102020000092FC37002B01D00021009A386801F0A3
:102030002FFF2900009BCB311A784F4BD3351A6004
:102040004B780A781B0213438A7812041A43CB7820
:102050001B061343494A1BBA13604B790A791B02CA
:1020600013438A7912041A43CB7931001B061343B8
:10207000434A1BBA13606B782A781B021343AA7871
:1020800012041A43EB781B0613433E4A1BBA136033
:10209000019A330213433C4A13603C4B22001B1B42
:1020A0009C4603293DDCB3089A0013005142B21A42
:1020B000032A46D1354AE018511A82784078120432
:1020C00000020243E05C043302430A600022FF2B5B
:1020D0004BDDF0222E4B12011A600F222D4B1A609D
:1020E0002D4A1368002BFCD00023224A2749136095
:1020F000091B321D0B191B68043A180A2370607003
:10210000180C1B0EA070E3700434002AF2DC80224D
:1021100010213B68D20501333B6093688B43936089
:10212000F7BD6346D578981893782D061B042B438A
:10213000157804392B43557804322D022B43036064
:10214000AFE7022A0AD1114AE05C511AE21852782C
:10215000120202430A6004339BB2B7E7012AB5D1E9
:102160000A4A521AE15C1160F5E7084959180A60F9
:102170000433ACE7000004403C0004403800044055
:1021800034000440300004400C00044000010440CE
:10219000040004401000044014000440F7B515008A
:1021A00080221C001023D2050091916807000B4388
:1021B00093600023654AD730136001F041FE9D23F0
:1021C0003E009B00F9583B00CA363200FC33002920
:1021D00000D07FE0586801F05BFE390032785C4B3C
:1021E000CB311A604B780A781B0213438A78AC46CD
:1021F00012041A43CB78281D1B061343554A1BBAF9
:1022000013604B790A791B0213438A7912041A432B
:10221000CB791B061343504A1BBA13604B7A0A7AD8
:102220001B0213438A7A12041A43CB7A21001B063D
:1022300013434A4A1BBA1360009A2B021343484ABD
:1022400013602200474B1B1B0093009BCE785B184A
:1022500001938B7836061B0433430E7804383343DE
:102260004E78043136023343019E33600328ECDCA0
:102270000321A808431C9B002940800003292BD17F
:102280003849E5185E18A9786D78E35C09042D02D9
:10229000294319433160030008330021FF2B2DDD52
:1022A000314B324919600F21314B19600123274905
:1022B0000B60304B19680029FCD006211B680B40CD
:1022C000042B20D080220020D20593680A318B4352
:1022D0009360FEBD01217DE7022908D121495D18E7
:1022E000E1184978E35C090219432960D3E7012921
:1022F000D3D11C495918E35C0B60CCE71948181876
:1023000001600433CAE7002310490B606346002BC9
:102310000CDC3B00FC335A68102101325A608022E9
:10232000D205936801208B439360D2E7009B9B18F2
:102330001B68190A13705170190C1B0ED3700423FB
:102340005B4291709C440432E0E7C04600000440C8
:102350003C00044038000440340004403000044095
:102360000C0004400001044004000440080F000079
:10237000100004401400044070B5061E19D002225B
:10238000614B9B799343012B13D1604B1A78FF2A41
:102390000FD15A78FF2A0CD19A78FF2A09D1DA781E
:1023A000FF2A06D11A79FF2A03D15B79FF2B00D1CE
:1023B000A7E0574B0C201A78012A08D00022554D6F
:1023C0001A702B781A00093A042A01D8212070BD0E
:1023D0005A1F012AFAD94C4CA07B042800D990E05E
:1023E000A279032A00D98CE0821E012A03D86288D0
:1023F0001F2A00D885E0002E61D0012E00D080E099
:10240000A288012AE2D0002B0AD10138032803D880
:1024100001F0D8FC151D19151F202E7001F0F8FCD5
:102420002B785A1E032A16D800253B4B1D60282303
:10243000237501F05DFEA8422ED0A580C6E70223D9
:1024400020202B70EAE7042322202B70E6E70323E9
:1024500021202B70E2E7073B012BB7D82F4B1B68DD
:10246000DB6A9B06B2D52E4B1A78002AAED1A27B2E
:10247000911E012901D9002AA8D1022280211A70B7
:102480002823284D89012878237501F0D1FE802169
:102490002878890101F0F4FD0123A380224B1B78E9
:1024A000002B0AD0FA228021204B92001B880902BF
:1024B0005A431C4B187801F06BFD002087E701F0B0
:1024C0007FFD2B78A680073B012B06D918482E707C
:1024D00001F0F6FC1E2001F09BFC114B114C1A7808
:1024E000002A06D080210022207889011A7001F08C
:1024F0009FFE01F02DFD80212078090201F098FE59
:10250000DBE7122063E7C046A60BFF1F6B09FF1F26
:102510001A09FF1F1C09FF1F4809FF1F4467FF1FFF
:102520002309FF1F1B09FF1F2109FF1F2C09FF1F84
:102530000010004010B5002901D001F011FD10BDC0
:10254000F7B5604B01919978A1239B004B435E4AFC
:10255000060014681022E418D6235B00E0583623E6
:10256000FF33E35C00279343222B41D1574B0F3AB3
:102570001A600760012501F03BFE019B1880E823EB
:102580005B00E35C002B01D0B34258DD0023504FC9
:10259000FB70AD33FF33E3581A68002A03D09B88E1
:1025A000DB439B071DD03823FF33E35C002B18D09F
:1025B0009B235B00E35C002B13D1D133FF33E35C3F
:1025C000B3420EDAA4235B00E15AE018090A023193
:1025D00001F0B6FD23000122FE33013E01351A87CA
:1025E000FA70E8235B00E35C002B2AD0A8B2FEBDA2
:1025F00003683D00002BBED081880430090A0231F7
:1026000001F09EFDD6235B00E3581F60B2E7230074
:10261000B133BA00FF339858013781880430090A72
:10262000023101F08DFDE8235B00E35CBB42EEDC90
:10263000E822F61AED1800235200A354A6E700275B
:10264000F1E7200001F034FD00281FD0002E1DDD31
:102650007319882647190193B600200001F058FC31
:102660005A30800020184068013581880430090AFA
:10267000023101F065FD200001F042FCA359013355
:10268000A351BD4202D0019B9D42E6D1114BE35CB8
:10269000002BABD095239B00E35C002BA6D00E4B08
:1026A000E15A0029A2D00D4AA35C994202D9013314
:1026B000A3549BE700231A212000A35401F0B0FC8F
:1026C00094E7C046300DFF1F3409FF1F001403407C
:1026D000E010FF1F5A020000720200005E020000BC
:1026E000F8B51D4B1D4F1A78002A10D1BA7B002A6D
:1026F00002D101321A7003E0032AFAD0022AF8D07C
:1027000001F0F6FC00220120154B1A70F8BD154BA4
:10271000154D1C68154B9E7801232B702878C0B28C
:1027200000F0CEFCBB7B002B0BD101F061FBA123A1
:102730009B007343E41883239B00E41823782B70D9
:10274000E4E7032B02D101F02BFDF0E70020022B80
:10275000DCD101F03DFDEAE71C09FF1FA60BFF1FBE
:102760002309FF1F3409FF1F490AFF1F300DFF1FF8
:10277000F0B587B00EAD2F780FAD2D780593AC4630
:10278000634614000E4D0CAA12782E7803930D9B0D
:10279000009201932200059B029701F071FB2E70BD
:1027A000012C01D0042C08D1802206498B88934348
:1027B000054A1278D20113438B8007B0F0BDC046A2
:1027C0001C09FF1F6C11FF1F7809FF1F0B001B3B2B
:1027D00070B504003020E02B0DD81300E025493BF4
:1027E000FF3B9BB2ED00AB4205D8034B20001982A2
:1027F0005A8201F08DFD70BD8410FF1F10B501F0ED
:1028000027FC054B00205B68052B04D9034A52685E
:10281000D20200D4980810BD00100040FCE100E096
:1028200070B501F0CDFB0D4B1B68FC33DC691D6AF4
:10283000FFF7E4FF6419844204D2094B01241B68AA
:10284000002B07D004220024064B1A70064A936915
:102850000133936101F07CFB200070BD4467FF1FD2
:102860009809FF1F2309FF1FFC0FFF1F70B50C4DB8
:102870002B68FC335C6A01F0A3FBFFF7BFFF2B68FA
:102880000025FC339B6AE318834204D2054B1B6886
:10289000AB4200D1051B01F05BFB280070BDC046B8
:1028A0004467FF1F9809FF1FD722044B92009B58D3
:1028B00010B5002B00D0984710BDC0460000FF1F88
:1028C000F0B587B001F008FAFFF7EEFFC54BC64C34
:1028D00004931B78022B45D1C44B1B68186A01F086
:1028E000CFFCC34BC34A1A60C34BC44A1A60A02230
:1028F000C34B52001A60049B187801F091FAC14949
:10290000C14801F03DFCC149C14801F039FC102229
:10291000C04BFF201A60802252031A60802292036B
:102920001A60802212041A6001F092FC012001F06A
:102930009FFAFA20400001F0CBFB582001F010FC78
:10294000B54801F0F5FA012001F042FB072001F043
:102950005FFCE26DB14B1A4084235B001343E365D7
:1029600007B0F0BD01F094FBAD4E0290322001F0B3
:1029700087FC33681B0628D43C2001F081FC0F2023
:1029800001F07EFC974B1B78012B00D113E18025D1
:1029900033682B4200D0A1E0636C03202B436364B7
:1029A00001F06EFC01F074FB029B0299C31A5A1EDF
:1029B000814200D81A009B4B1A608C4B19681E2369
:1029C0005343994A9B18CB618BE701F061FB80234D
:1029D000E26BDB0213430390E363E26D8F4B032052
:1029E0001A4028231343E36501F04AFC0320A56E37
:1029F00001F046FCA36E0320DB03DB0B019301F027
:102A00003FFCA76EED03FF03ED0BFF0B874AAB18EE
:102A1000C22B2ED8019B9B18C22B2AD8BB18C22BC5
:102A200027D8019B2A009D4200D21A00019B9D429B
:102A300000D91D003B00974200D21300BD4200D9CF
:102A40003D005B1B122B14D80C22336814209343D7
:102A500033603368764A1340336001F011FC08217B
:102A6000A36EE26DDB038A43E265724ADB0B1360FF
:102A700085E7032001F004FCA36EDB03DB0B059369
:102A800001F006FB039B0399C21A531E814200D832
:102A90001300694A93421BD9FF23356864492D0A04
:102AA0001D4032686B1C1B060A401B0C134333602D
:102AB0000C23326800209A43083B1343336001F033
:102AC000BFFA5E485E4BA840984205DCFEF73AFF2D
:102AD000019D0197059F99E75A48F7E700235A4E51
:102AE00033608023226CDB0213432364636C032076
:102AF0002B43636401F0C4FB3368013333608023EC
:102B0000626C5B021343636405230193E26D434BE4
:102B100003201A404D4B1343E36501F0B1FB08213C
:102B2000A26EE36D434F8B43E3653B6802394B4331
:102B3000D203D20B9A420CD89B1A3B2B0BD8E36DD5
:102B400043490B40E365636C0B406364414B1A607F
:102B500028E7D31AF1E7019B013BDBB20193002B7D
:102B6000D4D1E36D3A4A1340E365636C1340636468
:102B70003368042B07D9BFF34F8F374B374ADA60DE
:102B8000BFF34F8FFEE7636C0320AB43636401F038
:102B900077FBE26D214B03201A4028231343E365A2
:102BA00001F06EFB0822A36EDB03DB0B3B60E36DE1
:102BB0009343E3659AE70722E36B1340012B02D1AD
:102BC000002001F02DF9264D264AAB680220134063
:102BD000AB6001F055FB8023AA685B001343AB6038
:102BE000E0E6C0464A0AFF1F00F000404467FF1FAE
:102BF000000003400180063DBC0003403408000093
:102C0000A40003407102000014100040FFFF3F00C9
:102C10002810004000E100E03075000000FEFEFFDB
:102C2000C4F000402C67FF1F7206000091FCFFFFFC
:102C3000FF00FFFF3467FF1FE30C0000E880000087
:102C40005F361E0060361E009C45FF1F28000100F5
:102C5000FFFFFEFF3067FF1F00ED00E00400FA05F4
:102C60003CF00040FFFEFFFF694E336888331B686D
:102C700083F3088801F054FB00F018FC654B664AAA
:102C80001B68934207D0002001F0DAF90221634A61
:102C900013688B431360FFF713FE614B614C187888
:102CA000C0B201F0DDF90023A3600233A3605E4BE4
:102CB0000120236001F0E4FA0323A36001F0E8F9A6
:102CC000040001F0C5F9050001F0E2F9574B186066
:102CD00001F0E6FA564B1968621A531EA14200D25F
:102CE00013008022D203934201D39B029B0A3268D5
:102CF000D16AC90700D478E04E491C0C09689BB220
:102D00004C4359432402090A641803274A49FC32F8
:102D100093680A6849489B1A494A4A4E12684A49C8
:102D20009B18414A34609A183B400193036892080B
:102D30009C46019B0A6063440360042B03D9013263
:102D40003B400A6003600B684049E418200001F032
:102D50007FF83F4F3D493B68C3183B60200001931B
:102D600001F006F93B4C2068081838492060884279
:102D700005D9019B01333B6001F0FAF8216001F0B5
:102D8000AFF8354B1B78002B0ED001F061F931689C
:102D9000324B4A1B1B6812189A4233D2591A4919EE
:102DA000091A2F4801F0ECF92E4C237A002B0FD092
:102DB00001F04EF93168E3684A1B1218934224D996
:102DC000591A4919091A284801F0DAF9002323721F
:102DD000264B83F3088801F04BF9022001F018F824
:102DE000002001F02DF901F05BF9DC0199000234BB
:102DF000641A5900641A09214B438033CB40A4085C
:102E0000E41882E7FA218900CBE71949DBE7C046DD
:102E10004467FF1F0C0AFF1FB6412103100000404A
:102E2000490AFF1F14100040C4090000100AFF1FC8
:102E3000340AFF1F380AFF1F200AFF1F280AFF1F3E
:102E40001C0AFF1F2867FF1F240AFF1F71020000D2
:102E50006008FF1F2C0AFF1F1C09FF1FE408FF1F4B
:102E600000100040740BFF1F3C10004000000020C9
:102E7000DC050000A022054B92009B5810B5002BEA
:102E800001D0984710BD01F01BFAFBE70000FF1FBF
:102E9000A122054B92009B5810B5002B01D09847FA
:102EA00010BD01F00DFAFBE70000FF1FA222054B49
:102EB00092009B5810B5002B01D0984710BD01F02F
:102EC000FFF9FBE70000FF1FA322054B92009B5870
:102ED00010B5002B01D0984710BD01F0F1F9FBE7C8
:102EE0000000FF1FA422054B92009B5810B5002B39
:102EF00001D0984710BD01F0E3F9FBE70000FF1F88
:102F000070B501F0A5F8514B1860042000F080FF67
:102F100001F066F90400C30702D401F0A1F970BD05
:102F200000224B4B1A604B4B1878013804282CD8E0
:102F300000F048FF03231B1F2700200001F0E8F8E2
:102F40000128ECD0444C2378042B71D101F050F8C7
:102F5000002806D001F074F9582001F001F902238D
:102F60002370032000F054FFD9E7200001F0C8F8D7
:102F7000E6E7200000F094FFE2E7200001F078F996
:102F8000DEE7200001F0A4F9DAE701F0E1F805003E
:102F9000012808D1314B1B78053B012B03D82000B9
:102FA000FFF768FFCEE72C4B1B78022B01D0052BD7
:102FB00020D1022D28D12A4B9B7BAB431CD1200072
:102FC000FFF766FF254B18780128BBD16405B9D4FB
:102FD000234925224B7B034205D1233A13405A4211
:102FE000534126331A000B7D9342ABD9322000F0B7
:102FF0007FFFA7E7022D07D1184B1B78052B11D1B6
:103000002000FFF753FFDDE7012D0BD1012B03D18A
:103010002000FFF759FF95E7062B03D12000FFF7AB
:1030200061FF8FE7200001F04BF9022D8AD1C9E73B
:10303000032B04D10B4B987C00F04AFF91E7072B40
:103040008FD1094B987B01F0BBF88AE79C09FF1FE1
:103050009809FF1F9009FF1F2309FF1F1C09FF1F6D
:10306000A60BFF1FBC0BFF1FD40BFF1FFA210A4B3F
:103070000A4A49001A640A4A5A500A4A04395A50FC
:10308000094A08319A64094A5A50094A5C315A502F
:10309000084ADA667047C0460000FF1F7127FF1F0D
:1030A0006D28FF1F2128FF1F7923FF1FE126FF1F27
:1030B000011EFF1FD51DFF1F10B500F06BFE10BDD8
:1030C0008023F7B59C46264B264F01932649274A75
:1030D000274D284C284B02281AD1604638600868D2
:1030E000264E304080263603304308600199097827
:1030F000002909D11660224A2A60224A2260E02271
:1031000019689143A03A1BE08021C9021160F2E7DF
:1031100066463E600F68194E3E408027FF023E43E0
:103120000E600199097800290DD1176001280ED190
:10313000154A2A60154A2260E02219689143C03A74
:103140000A431A60F7BD802189021160EEE7E02191
:103150000F4A02432A600F4A22601A688A43F0E746
:103160004B0AFF1FE0000340D800034090000340DB
:10317000000003405000034040000340FFFFE3FF16
:103180000280063D804508220180063D80660822B7
:103190000080069880550822F8B51E4B80261A68D4
:1031A000002014003440324232D11A681A4F3243A0
:1031B0001A6001223B68063093433B6001F060F8DF
:1031C0000122164D2B681E432E603B680A261343CE
:1031D0003B608027BF00124B1B683B4211D1013E70
:1031E000F6B2FF2E09D17E220E4B1C682B68E40B31
:1031F0001440934323432B6005E0082001F040F87E
:10320000E9E7002EEFD180222B68600893432B6002
:10321000F8BDC046C4F000405CF0004018F000402B
:1032200068F0004060F0004010B500F0F1FE0121B0
:103230005820034A00F054FFFFF7AEFF10BDC04610
:10324000600AFF1F10B578220021034800F0B0FE8D
:1032500000F0D6FD002010BD4C6AFF1F70B50400C1
:1032600000F0AEFE00230C200B4A010059438D18DC
:10327000515C00290DD0A14208D1012300246B70BC
:1032800001F03EF800F064FE200070BD01330A2B0F
:10329000EBD11224F6E7C0464C6AFF1F70B504005C
:1032A00000F08EFE002319001D000D4A1078002842
:1032B00006D0A0420CD1557001310C320A29F5D14B
:1032C000002B0AD100F09CFD00F042FE002070BDF2
:1032D0005078461EB0411B18EEE701F011F8F3E7F5
:1032E0004C6AFF1FF7B504000C20002384460E4DE6
:1032F000019267465F43E85D7E19A04212D0002824
:103300000BD10A4B9C4662461B7808331370019B15
:1033100070707C557160B360FEBD01330A2BE8D13B
:103320000320F9E70720F7E74C6AFF1F486AFF1FF1
:103330008020F8B5484BC0051B68C1248360474B0B
:10334000FF251A68012313434361454BA4001A6803
:10335000444B40211A60444B1A68444B1A60444B5A
:103360001A59AA431A51C52292009E58AE433143BE
:10337000802699509F583F49F6010F403E439E508A
:103380009E5880273602360A3043985080201A59BA
:1033900000020A4002431A5104341A59364E3F04BF
:1033A000324080263A431A511A5936061202120A3E
:1033B00032431A5108341A5980260A4002431A51DE
:1033C000C32292009F58B446AF4337439F509F5843
:1033D000294E0F4007439F509F58374080263604A0
:1033E000374380269F509F5836063F023F0A374397
:1033F0009F50C0221F59AF433A431A511A59120223
:10340000120A1643C6221E5192009C58AC436546D0
:103410002C439C509C5800250C4020439850C720BA
:1034200080001A58154C1140C02212020A431A504B
:10343000134B1B78DB08AB4201DC0020F8BD23787E
:10344000002B06D0A368002B00D0984701350C3420
:10345000EEE71220F2E7C0463446FF1F3046FF1F5A
:10346000B0F00040446AFF1FB4F00040406AFF1F04
:1034700000E100E0FF00FFFFFFFF00FF4C6AFF1FBD
:10348000486AFF1F030010B51F2809D80722002033
:103490001340072404490A78A24313430B7010BD5C
:1034A00000230620F5E7C046486AFF1F034A044987
:1034B000136800200B4013607047C0461CF00040AA
:1034C000FFFFC1FF054B06491B780A6805485B07EB
:1034D00002401B0B134300200B607047486AFF1F1C
:1034E0001CF00040FFFFC1FF70B50C25FFF7EAFF9D
:1034F0000A4B1C780A4BE4086543ED18002C01D1F7
:10350000200070BD2B78002B06D06B68002B00D0FC
:103510009847013C0C3DF1E71220F2E7486AFF1F93
:10352000406AFF1F1FB5002102220B00019100918C
:10353000052000F0F5FD02230B490A681A42FCD170
:1035400020230393039B5A1E0392002BFAD1074AB0
:103550001368002BFCDA0B246C442000012100F0DE
:10356000AFFD207804B010BD90C8004000C80040F6
:1035700013B504000A4B0193019B002B01D11120CC
:1035800016BDFFF7CFFF23000340044205D00520FE
:1035900000F076FE019B013BEDE71800F0E7C04626
:1035A000FFFFFF0707B500F00BFD80220821D205C1
:1035B000936A0191002B01D10739916202210C4AD3
:1035C00011600199481E01900029FAD10331116060
:1035D000053101910199481E01900029FAD111602D
:1035E000002B02D18022D205936200F0B1FC07BD0E
:1035F00000C00040F0B52D4C89B02378002B4FD18E
:10360000FEF780F902232A4F03903A681A42FCD150
:1036100020230693069B5A1E0692002BFAD1254EB4
:103620003368002BFCDA0120FFF7A2FF011E02D055
:10363000112009B0F0BD030003220190009005ADF8
:103640009F2000F06DFD0321280000F039FD0223CA
:103650003A681A42FCD120230793079B5A1E07920F
:10366000002BFAD13368002BFCDA0120FFF780FF32
:103670000028DDD10398FEF759F9AA786B78110478
:103680001B020B4329780B4363601300113B0A496B
:10369000052B07D801239340A3600B6001232370FF
:1036A0000020C6E780231B03F6E7C0461C46FF1F29
:1036B00090C8004000C800409808FF1F1E4B30B55E
:1036C0005A6818781D4B85B0D31859424B410121D7
:1036D0000093002300F04CFD194B1A4A02259A630F
:1036E00000221A6510325A658022C4219D65164B4E
:1036F0001648D202DA6789004258154B80241A40D6
:1037000080231B0413434350642341200393E405A7
:1037100000F006FA402000F003FA6562039D6B1E7C
:103720000393002DFAD103236362FFF73BFFA562E9
:10373000FFF760FF05B030BD2846FF1F95FFFEF77D
:1037400000C80040050001FF04E100E000E100E0E6
:10375000FFFF00FFF0B585B00700FEF7D3F80223A6
:1037600005002D4C22681A42FCD120230093009BB7
:103770005A1E0092002BFAD1284E3368002BFCDA37
:103780000120FFF7F5FE002803D01124200005B02A
:10379000F0BD234B2360022322681A42FCD1202370
:1037A0000193019B5A1E0192002BFAD13368002B22
:1037B000FCDA0120FFF7DCFE0028E6D1194B1F6080
:1037C000022322681A42FCD120230293029B5A1E34
:1037D0000292002BFAD13368002BFCDA0120FFF7AC
:1037E000C7FE0028D1D1104B2360022322681A4261
:1037F000FCD120230393039B5A1E0392002BFAD182
:103800003368002BFCDA0120FFF7B2FE041EBCD1A6
:103810002800FEF78BF8B9E790C8004000C80040C8
:1038200001000006A8C800400180000110B500207A
:10383000FFF790FF10BD000010B5064B18705960DF
:10384000FFF73CFF00211320034AFFF74BFD002048
:1038500010BDC0462846FF1FBD36FF1FF0B504004F
:1038600085B003920291FEF74DF8882263035B0B4B
:1038700052051A438023DB059D6A8023274F00925F
:10388000BA68002601901B039A420CD9F82326003F
:103890001B041E401C4206D08022214B52025E6255
:1038A00019680A431A60002D0BD100F089FB02222F
:1038B0001C4B1A608023DB055A62013A9A6200F0C1
:1038C00047FB0023039A934220D1002D0AD100F038
:1038D00077FB144B03221D608023DB055A629D6237
:1038E00000F036FB8023BA681B039A4208D9002EE9
:1038F00006D000220A4B0C495A621A680A401A6024
:103900000198FEF713F8002005B0F0BD009A029967
:10391000D2181278CA540133D4E7C0461C46FF1FA0
:1039200000C8004000C00040FFFFFEFFF0B587B0B8
:10393000029103920400FDF7E5FF019000F040FBC7
:10394000802302250122234EDB0535605D629A62E9
:1039500000F0FEFA204F3B682B42FCD12023049359
:10396000049B5A1E0492002BFAD11C4D2B68002B8D
:10397000FCDA0120FFF7FCFD002802D0112007B07F
:10398000F0BD2000039A029900F06AFA02230400B5
:103990003A681A42FCD120230593059B5A1E0592D2
:1039A000002BFAD12B68002BFCDA0120FFF7E0FD99
:1039B000051EE3D100F004FB80230322DB05356004
:1039C0005A629D6200F0C4FA0198FDF7AFFFE0B2C1
:1039D000D5E7C04600C0004090C8004000C8004085
:1039E000F0B5802489B00600FDF78CFFE405A36ADA
:1039F00002250393029000F0E3FA0123304F3D606B
:103A00006562A36200F0A4FA2E4C23682B42FCD11D
:103A100020230593059B5A1E0592002BFAD12A4DAF
:103A20002B68002BFCDA0120FFF7A2FD002803D051
:103A30001124200009B0F0BD244B2360022322682A
:103A40001A42FCD120230693069B5A1E0692002B95
:103A5000FAD12B68002BFCDA0120FFF789FD021E4A
:103A6000E6D11B4B03211E60030001900090202033
:103A700000F056FB022322681A42FCD12023079350
:103A8000079B5A1E0792002BFAD12B68002BFCDAF9
:103A90000320FFF76DFD041ECAD100F091FA8023C8
:103AA0000322DB053C605A629C6200F051FA039BE2
:103AB000002B01D1FFF776FD0298FDF737FFB8E73D
:103AC00000C0004090C8004000C80040010000064F
:103AD00094C8004007B5000201910422000A01A920
:103AE000FFF724FF0EBD000073B5050005240B4A47
:103AF000A3005B429B1819686B46DE1D300000F086
:103B000097FA022804D133782B55013CEFD276BDC9
:103B1000052CFCD00128FAD10230F8E71409001175
:103B20001F2807D8012380228340D20591680B43C8
:103B3000936070473F2808D80123802220388340B3
:103B4000D20551690B435361F3E75F28F1D8012394
:103B5000802240388340D205116A0B431362E8E7A4
:103B60001F2807D8012280218240C9058B68934312
:103B70008B6070473F2808D801228021203882407E
:103B8000C9054B6993434B61F3E75F28F1D80122E4
:103B9000802140388240C9050B6A93430B62E8E7F5
:103BA0001F2810D880230200DB05153A1968012A66
:103BB00006D820229143196019680A431A60704799
:103BC00001228240F6E73F2811D880230200DB055E
:103BD000353AD968032A06D810229143D960D968AA
:103BE0000A43DA60EBE7012220388240F5E75F28DC
:103BF000E5D842238022181A413B8340D205516AFE
:103C000099435162516A0B435362D8E710B50400DF
:103C1000012813D1A022184992050B685B015B09AA
:103C200013430B60154B164A19681140154A0A4395
:103C30001A60402219680A431A6010BD0028FCD19E
:103C400001000A2000F09CF921000B2000F098F9F7
:103C5000C0220A4B920019680A4340211A601A6870
:103C60008A431A60B022044912060B685B015B09A3
:103C700013430B60E1E7C04614F000401CF0004025
:103C80007F00FEFF80FD010072B6074A1368013312
:103C900013600422054B1A600023054A136080223A
:103CA000D2055360FEE7C0467808FF1FC0F0004011
:103CB000C4F00040044B054A1A60054B1A6000220C
:103CC000044B1A607047C046140AFF1F841E000090
:103CD000380AFF1FC4F000400023034A1360034A60
:103CE0001360034A1360704754F0004040F10040F5
:103CF00044F10040002310B5184C8AB000930193A2
:103D00002378012B27D06946012000F019F90028FB
:103D100017D1009B12490293019B06AA0393114BF2
:103D200002A81B680493104B1B68059300F078FAF7
:103D300010220E4906A800F0BBFA002804D1FF2388
:103D4000237000200AB010BD0123094A074902A8C8
:103D5000237000F065FA0120F4E7C0464867FF1FB2
:103D600010290011082900110C2900112029001127
:103D70004C67FF1F13B501246946012000F0E0F8ED
:103D8000034B00940193FFF7B5FF200016BDC0461A
:103D9000BB0B000010B5FFF79FFFFFF7EBFF0028FC
:103DA00002D0024B984710BDFEE7C046E1A20000DA
:103DB00002B4714649084900095649008E4402BCC4
:103DC0007047C04602B4714649084900095C490081
:103DD0008E4402BC7047C04603B471464908400097
:103DE0004900095A49008E4403BC70470000000096
:103DF00001B40248844601BC604700BFE9F60000F8
:103E000001B40248844601BC604700BFADAE00006B
:103E100001B40248844601BC604700BF1907010095
:103E200001B40248844601BC604700BFEDA5000014
:103E300001B40248844601BC604700BFF9ED0000B0
:103E400001B40248844601BC604700BF89440000B9
:103E500001B40248844601BC604700BF090E00005F
:103E600001B40248844601BC604700BF957301005D
:103E700001B40248844601BC604700BF69110100DB
:103E800001B40248844601BC604700BF9D6A00003F
:103E900001B40248844601BC604700BF21440000D1
:103EA00001B40248844601BC604700BF05340100EC
:103EB00001B40248844601BC604700BFA1AF0000C6
:103EC00001B40248844601BC604700BFC1A50000A0
:103ED00001B40248844601BC604700BF4DF90000B0
:103EE00001B40248844601BC604700BFD5440100CC
:103EF00001B40248844601BC604700BF613701003D
:103F000001B40248844601BC604700BF59760100F5
:103F100001B40248844601BC604700BFD9B000002C
:103F200001B40248844601BC604700BFF9A6000006
:103F300001B40248844601BC604700BF8D110100F6
:103F400001B40248844601BC604700BFE1AC0000F8
:103F500001B40248844601BC604700BF9DA900002F
:103F600001B40248844601BC604700BFE9D40000A8
:103F700001B40248844601BC604700BF090E00003E
:103F800001B40248844601BC604700BFBDA30011D4
:103F900001B40248844601BC604700BF8B52010057
:103FA00001B40248844601BC604700BF85B70011D8
:103FB00001B40248844601BC604700BFB70E000050
:103FC00001B40248844601BC604700BF75A90000E7
:103FD00001B40248844601BC604700BFE5120100FD
:103FE00001B40248844601BC604700BF51B80000DC
:103FF00001B40248844601BC604700BF01D70000FD
:1040000001B40248844601BC604700BFE9270000B4
:1040100001B40248844601BC604700BFED6801005E
:1040200001B40248844601BC604700BF53B9000098
:1040300001B40248844601BC604700BF99380011B2
:1040400001B40248844601BC604700BF016C010016
:1040500001B40248844601BC604700BFC95C01004E
:1040600001B40248844601BC604700BF89140100C6
:1040700001B40248844601BC604700BF7997000044
:1040800001B40248844601BC604700BF0D520100E4
:1040900001B40248844601BC604700BF156B0100B3
:1040A00001B40248844601BC604700BF855201004C
:1040B00001B40248844601BC604700BF71B00000F3
:1040C00001B40248844601BC604700BF3D71010055
:1040D00001B40248844601BC604700BF851201005C
:1040E00001B40248844601BC604700BF016701007B
:1040F00001B40248844601BC604700BFA9D8000053
:1041000001B40248844601BC604700BF0934010085
:1041100001B40248844601BC604700BF013401007D
:1041200001B40248844601BC604700BF496D0100EC
:1041300001B40248844601BC604700BF85C100004D
:1041400001B40248844601BC604700BFC1150100AC
:1041500001B40248844601BC604700BFDD0C010089
:1041600001B40248844601BC604700BF79120100D7
:1041700001B40248844601BC604700BFC56D010020
:1041800001B40248844601BC604700BF2D6C0100A9
:1041900001B40248844601BC604700BFE90B01003E
:1041A00001B40248844601BC604700BF75F80000B6
:1041B00001B40248844601BC604700BFE94C0100DD
:1041C00001B40248844601BC604700BFC1F700004B
:1041D00001B40248844601BC604700BF19FA0000E0
:1041E00001B40248844601BC604700BFBD0B01001A
:1041F00001B40248844601BC604700BFCD0C0100F9
:1042000001B40248844601BC604700BFBD5C0100A8
:1042100001B40248844601BC604700BFF90D0100AB
:1042200001B40248844601BC604700BFDD3F000086
:1042300001B40248844601BC604700BFB35201008C
:1042400001B40248844601BC604700BF6DF600001F
:1042500001B40248844601BC604700BFED6B010019
:1042600001B40248844601BC604700BFDD0A01007A
:1042700001B40248844601BC604700BFF535010027
:1042800001B40248844601BC604700BF01890000B8
:1042900001B40248844601BC604700BF8937010071
:1042A00001B40248844601BC604700BFC1660100FA
:1042B00001B40248844601BC604700BFCD4C0100F8
:1042C00001B40248844601BC604700BFE917010001
:1042D00001B40248844601BC604700BFF9350100C3
:1042E00001B40248844601BC604700BF6D0B010069
:1042F00001B40248844601BC604700BF8D820000C3
:1043000001B40248844601BC604700BF21A90000F7
:1043100001B40248844601BC604700BF116E000032
:1043200001B40248844601BC604700BFC9A900002F
:1043300002000000C6C00011010000007CBE001198
:1043400002000000C2C00011010000007043FF1F06
:104350000200000084BE0011010000008C64FF1FF9
:1043600002000000C0C00011030000000064FF1F35
:104370001200000002000000C6C000110100000091
:10438000C0BE001102000000C2C000110100000008
:10439000BDBE001102000000CABE001103000000F3
:1043A0003B64FF1F02000000C0C0001103000000BA
:1043B0005064FF1F02000000C2C000110100000095
:1043C000BCBE001102000000C8BE001103000000C6
:1043D0001164FF1F02000000C0C0001103000000B4
:1043E0003264FF1F02000000C6C00011010000007F
:1043F00000BF001102000000C2C000110100000057
:10440000B944FF1F0200000012BF001101000000AC
:10441000FBBE001102000000C2C00011010000003C
:10442000B844FF1F0200000010BF0011010000008F
:104430005864FF1F02000000C2C00011010000000C
:10444000B744FF1F020000000EBF00110100000072
:10445000EBBE001102000000C2C00011010000000C
:10446000B644FF1F020000000CBF00110100000055
:10447000E6BE001102000000C2C0001101000000F1
:10448000B544FF1F020000000ABF00110100000038
:10449000E1BE001102000000C2C0001101000000D6
:1044A000B444FF1F0200000008BF0011010000001B
:1044B000DCBE001102020202020200000000000045
:1044C0000D0C0000614D0011274D001154BF00116B
:1044D00090011D0018001800FFFF070102030405EA
:1044E00006020106000000000000000000000000BD
:1044F00000000000000000000000000000000000BC
:104500000300000002000000C6C00011010000000E
:10451000D4BF001102000000C2C000110100000061
:104520007445FF1F02000000DEBF00110100000003
:104530008664FF1F02000000C0C0001103000000DD
:10454000F066FF1F02000000C2C000110100000061
:104550007445FF1F02000000DCBF001101000000D5
:104560008864FF1F02000000C0C0001103000000AB
:10457000E866FF1F126C6C6C0000000000580040E1
:10458000151600000001000000000111FFFF0000EF
:1045900050485936000000000000000001000000F3
:1045A00065BF00110B000500F7000000B4000028F3
:1045B000002800283075A000A000A000A00000087E
:1045C0000008E001F00010001000100010001000C2
:1045D000100050005000500010001000D0070000E4
:1045E000000000000F0001000500307507001000FA
:1045F000010081FF00000000FF000000A575001110
:10460000AD7300113D710011FFFF0100FF000000BC
:10461000C19F00113D9D0011559C0011000000003C
:104620000000000000000800040000003B0001083A
:104630005902E00188212800FF000000020000006C
:10464000C6C00011010000008CC100110200000072
:10465000C2C0001101000000B946FF1F02000000A7
:10466000BEC0001101000000046BFF1F020000002B
:10467000C2C0001101000000B846FF1F0200000088
:10468000BCC0001101000000B646FF1F0200000080
:10469000C2C0001101000000B446FF1F020000006C
:1046A000BAC0001101000000AC46FF1F180018003E
:1046B0001D00900102000003020200000200000041
:1046C000C6C0001101000000A0C1001102000000DE
:1046D000C2C0001101000000FC46FF1F02000000E4
:1046E000B8C000110000000000000000020000003F
:0E46F000C0C0001103000000246BFF1F20FF5C
:040000051FFF184180
:00000001FF
